:020000040000fa
:080000000002040000000000f2
:020000040000fa
:10040000ef4421000e7f24000e0188000000000050
:100410000c000700601e23000100200011000700ef
:10042000000020000000e000020032000000020096
:100430000000000030440200000000000040da002c
:100440000000fe004440a900606620000000e000bb
:100450000300320000002000a00188004440a800f2
:100460000000060091018800800078000000eb0089
:1004700015003700e280400032a0b4009101ba00bc
:10048000e280400032a0b4009102ba00e280400055
:1004900032a0b4000002eb00472bde00f507b200eb
:1004a000602ce10004003a000059eb008301e900f0
:1004b000fdff3e00040037006128e100010032002a
:1004c0000082eb00040007001101ba000200e00006
:1004d000e8ff3a00000006003159ba008301e90044
:1004e0000c0032002159ba008301e90008003200f3
:1004f0000400e00003003a00e280400032a0b400b3
:10050000f5ff370011d9ba008301e900faff3a007c
:100510008100e800e180400032a0b4000000060045
:1005200048210400000000005821040000000000e1
:100530006821040000000000782104000000000091
:100540008421040000000000962104000000000047
:10055000e6210400000000006c22040000000000fe
:10056000f42104000000000030220400000000001c
:10057000ae240400000000006c260400000000000f
:10058000cc27040000000000442304000000000009
:100590000e280400000000003228040000000000c3
:1005a00048280400000000005c280400000000004f
:1005b00072280400000000000040da000000fe0085
:1005c000800078001106b100030035009101b100f0
:1005d00001003c000050a100000006000003b10033
:1005e0000b0035009000b100080034008000b1001d
:1005f000070035009001b100040034007000b10024
:10060000030035009001b10001003c00100005001e
:10061000000005000a00fa0080017800e20f500097
:1006200028003e0060a28000e10f50000800320068
:10063000802320000000e000050032000423200099
:100640002523200046232000800178000400370085
:1006500004222000252220004622200083222000a0
:10066000144090000004e000040035008009eb0015
:10067000144090000074a0001042980015409000b3
:100680000028a30003003a00154090000024a000b9
:10069000904298008001eb00070037001540900061
:1006a0000008a300fdff320063c078000000fb00db
:1006b000000b78008301e800828f5100f7ff3a00b9
:1006c0000800370030002000b0bf9f00c3bf9f006c
:1006d000d1bf9f00e2bf9f006a80570000c0da00d0
:1006e0006fb99700020078000080fa000000060051
:1006f0000001be00200107000470a70003f0a10064
:100700006509b100160032000d0035006828e100cf
:1007100006003500f0ff2f00f1ff27000300e00086
:1007200013003b000100280000000500000040000d
:10073000818048008502e900fcff3a00080037008c
:10074000f88f420002003c008000eb000000050032
:100750008100d1000080d3008502e800fcff3a0050
:100760000300e00002003b0060001000e080180081
:1007700000000600889fbe008a9fbe000105780029
:100780000100e0000400350008003c000000e0002b
:10079000200032000500370060001000e0801800e3
:1007a00002003b0001f02c001a0037000004be00dc
:1007b0006011b8006b0920000982cf0002003900e7
:1007c0000882cf000441b000694252000e0032009e
:1007d00008003b0082817100610164008904d1003e
:1007e0000884d3008b05e8000442e800f9ff3a00d2
:1007f000050037000804440089844c008b05e9009b
:100800000442e900fbff3a00f00007000af0a700ed
:1008100001f0a0004f05be004f04be00000006001e
:1008200003f0a200889fbe008a9fbe008c1f780044
:100830000c010700130133006450e1004f00320047
:100840006420e1005200320003826c0007003b008c
:100850000905d0000306d000820f54000c065d008d
:100860000200390002003200890178000306780096
:100870008582550004003d000003fd008103fd005a
:100880008502ea008b854200840f720002003b0063
:1008900060001000e08018006011b8000005eb0057
:1008a0007a28e1000a00390006007800c75ddd0003
:1008b000f707b200878075002d0037008281710034
:1008c0000a017800610560008180d1000080d300ba
:1008d0008502e900f9ff3b000604400087844800d8
:1008e00002003b0060041400e0841c000988a3009f
:1008f000070032008a817100828171006101640009
:100900008904d1000884d3008b05e8001700370064
:100910000978a30013003a000b00e0001300340034
:100920008b05e9000804440089844c000a447400e3
:100930000978a3000d003a000b00e0000700340026
:100940008b05e9000804440089844c0001003a004a
:100950000b0020000978a300f7ff32000001eb0034
:1009600002003700828171000a01780097000700b9
:100970000cf0a70001f0a000cb0037006420e100dc
:1009800002003a00838f6c00cb0033000801be00e8
:100990000200be00c4003700889fbe008a9fbe00d0
:1009a0008c1f7800af000700b600330003866c0090
:1009b0006450e100240032006420e100270032008e
:1009c0006150e100220032006120e100210032008c
:1009d0008b854200eb07b1000134b800003ab80043
:1009e0000804420089844a00013ab8000030b80087
:1009f0008880400009014a000400330000004000e4
:100a000081804800020149008b05e900c909dd0029
:100a1000830170000100320013002000c814de00c2
:100a20004814dd004709de001200b200c808de00ed
:100a3000088470006500070001f0a1000cf0a70019
:100a400001f0a000980037006120e1009a00320018
:100a50000801be000200be00f7ff37006150e10050
:100a6000fcff3a0094003700889fbe008a9fbe00ba
:100a70008c1f78007b0007008200330003866c0027
:100a80006450e1002e0032006420e10033003200a7
:100a90006150e1002f0032006120e100310032009e
:100aa00085855500eb07b0000900200008042000f0
:100ab000050037000804440089844c000a00310016
:100ac0000603430087834b000001530081815b00d4
:100ad000f8ff33000203be000800a0000804440031
:100ae00089844c00f6ff3900c639dd0083017300ac
:100af00001003200130020008904d1000884d300d3
:100b00000998a300050032000800a7000300a00018
:100b10008904d1000884d3008b05e8008904d10042
:100b20000884d3000001eb000281d20027000700f7
:100b300001f0a1000cf0a70001f0a0005a0037005e
:100b40006420e1005c0032000801be000200be002b
:100b5000f7ff37006120e100570032006000b80065
:100b6000f3ff37000000200001f82700f0ff3700f6
:100b70001400200053003700c70ade00f107b2005e
:100b8000f50fb20008003200e1cf4200020032004f
:100b90000170a00024000500810f700001003200e8
:100ba0000408050044000500810f700002003a00af
:100bb000140005008502e9000000400081c04800e3
:100bc000fcff3b000170a000240005008100200014
:100bd000618055000b003d000b00200061fe2f00de
:100be0000100e1001d003400828171006101640098
:100bf0008904d1000884d3000000e800faff3a001d
:100c000071002000610064000300700002006000b9
:100c10000900320061044400e0844c000988a5000a
:100c2000050032008b05e8006808e10002003a0088
:100c30008904d1000884d300f20f20000258e1009b
:100c400005003d00c75ddd00f907b2008980750031
:100c500008007800000006000bf827008b007800e1
:100c6000000005000004be00c3ff07000003be0033
:100c70000405be000200be00bfff0700844f7500e0
:100c8000000006000200be006450e10005003600ce
:100c90006420e100020036000968a30001003a0068
:100ca0000800be000160a0004f0678004f05be009e
:100cb0004f04be0000000600f0ff2f00f1ff2700e8
:100cc000f9ff3700889fbe008a9fbe00841f78000e
:100cd000e4ff07004f00780011003300f0ff2f0001
:100ce000838f6c0006003b00040565000a00a70026
:100cf0000800370009f0a6001000200008003700a7
:100d0000820f5400838f5c00030039001000200024
:100d100001003e000000200009f0a7000000ea00ea
:100d20004f05be004f04be000000e00000000600ba
:100d3000881f7800000478005001be004000be000b
:100d40000400400085804800060149008781490071
:100d5000009cbe000294be000400e1000588e10092
:100d60000690e1000798e1000200310068004400ad
:100d70001008e8004f04780000000600f4874700e0
:100d8000889fbe008a9fbe008c9fbe008e1f780089
:100d90000205be000004be00d4b79f00e5b79f0067
:100da000f6b79f0087bf9f000000eb00c0b79f0011
:100db000b0b79f00a0b79f0090b79f0080b79f007b
:100dc0000d042000bfb097004fb097000001400015
:100dd0000000e0000f003d004f08de000000710041
:100de000c0b79f009e00070001003d0012002000d8
:100df000a100070001003d0012002000a60007002e
:100e0000b1000700b60007000f004000c8ff070050
:100e1000220037004f08de0000067100ccb79f00ab
:100e20008f00070001003d00120020009200070023
:100e300001003d001200200097000700a2000700fb
:100e40000fb297009fb297002fb39700bfb39700e0
:100e5000a90007000000520081805a0002015b00d7
:100e600083815b0080b79f0091b79f00a2b79f006e
:100e7000b3b79f000007eb009f0007000020e100d0
:100e800001a8e10002b0e10003b8e1000100310077
:100e90001e0020000e005600c0b79f004fb2970002
:100ea0000400e000070035001000200001002000d1
:100eb0006011b80008047000898470000a05710090
:100ec0008b8571008d06e900beff3a000400e0004a
:100ed00003003d00820007000f00400094ff070060
:100ee0004fa897000000e00004003a000fb49700fc
:100ef0009fb497002fb59700bfb5970094000700e7
:100f00004f0778004f06be004f05be004f04be00dd
:100f10004f01b10000000600881f78001800200073
:100f2000881f780095ff07008f87e9004f0478003d
:100f300000000600801feb0090ff07008f87e9008c
:100f400000000600889fbe008a9fbe008c1f7800ac
:100f50006e00070007003d0073000700e00f5b0014
:100f6000e08f5b0007003d00320007000006eb0049
:100f7000040037003400070002003d002a0007008b
:100f80001c00200072000700e3ff07000203be0000
:100f90000002be000c00e000010032002200070049
:100fa0000400be000601be004f0678004f05be00db
:100fb0004f04be0000000600889fbe008a9fbe004e
:100fc0008c1f78005100070005003d005600070007
:100fd000e00f5b00e08f5b0006003d00040037007f
:100fe0001900070003003d006000b8006011b80060
:100ff0001000070056000700ceff07000203be00e6
:101000000002be000c00e0000100320006000700f4
:101010000400be000601be004f0678004f05be006a
:101020004f04be00000006006000b8006011b80068
:101030000000370004025000858258000603590062
:1010400087835900000006000006eb00e00f520005
:10105000e08f5a00e00f5b00e08f5b0000000600ad
:101060000180400090b79f000001eb008fb0970017
:101070000100e000000006000200700090b79f0031
:101080000180400080b79f000001eb00ffa897009f
:101090000100e000000006000200700080b79f0021
:1010a000018040006faa9700cf20de000100700091
:1010b000f0af9f0004024200250007004f18de0039
:1010c0000002720000000600e4af9f000804440024
:1010d00089844c000a054d008b854d0000000600f8
:1010e0003fb29700cfb297005fb39700efb397007e
:1010f00000fe2f00000006003fb09700cfb0970021
:101100005fb19700efb19700000006000205be0036
:101110000004be00e00f5000e08f5800e00f5900bf
:10112000e08f5900000006006000b8006011b800b0
:1011300008045000898458000a0559008b8559001d
:101140001c002000e00f5200e08f5a000000060053
:101150000800be000a01be00000006002800fa00d8
:10116000889fbe008a9fbe008c9fbe0003866b00d6
:101170000c0207000028a30064003a000128a30025
:1011800067003a000008a30062003a000108a300cb
:1011900065003a001e009000be08900081064000e5
:1011a000ed3fb100f4805700ee019000111ab80035
:1011b0008e099000311bb8009e099000311cb800c8
:1011c000511db800f485570046000700fe0190004d
:1011d0003a0007008b85e8003e0007008e0990006a
:1011e00040000700ee019000340007008b85e80006
:1011f000380007008e099000400007009e0990000b
:101200001b18b800890440000a854800fe019000c0
:10121000340007008b85e80038000700ee019000dd
:10122000300007008e0990001b18b80089044000a8
:101230000a8548000a98a30008003a000402420008
:1012400085824a0006034b0087834b0008044c004c
:1012500089844c000a054d008d06e90084827200e5
:10126000850273004c3add008502720001003200f5
:1012700015002000443ade001400b2004538de00bc
:10128000cb45dd000b007000c540de00cb4ddd001e
:101290008b8070004549de00cb55dd000b017100ed
:1012a000c551de000d037800d701070003f0a1004f
:1012b0000cf0a70003f0a000ce0137001b18b80007
:1012c0008502400006834800e0834b0060044c0028
:1012d000070037001b18b80006034000878348004a
:1012e000faff37001b18b800870340000884480045
:1012f000e0844c0060054d00000006001b18b8009b
:101300000804400089844800faff37000108a30060
:10131000b5013a005800be005801be00e3ff370097
:101320000008a300b0013a0009047800f9ff370073
:101330008103780010fe07000001be006000b800c5
:101340000478a30013003a006220e10015003e007b
:101350000d0039008301d1000281d3008180d300c8
:101360008301d1000281d3008180d3008301d100a9
:101370000281d3008180d3000538b000c42add008b
:10138000f300b2008381720007f0a70003f0a00011
:1013900000000600f3ff2700f2ff2f006110b900e4
:1013a000fbff370003ff2700f7ff37008f1fd10037
:1013b000c10107008f87e9000000e000000006007f
:1013c000801feb00bc0107008f87e9000000e000f0
:1013d000000006001400fa00889fbe008a9fbe002d
:1013e0008c9fbe000005be000206be0068004700dc
:1013f0000c90be000a90be00d80107006400e10016
:101400001a00320016003e006100e1001a003200ae
:101410006e049000fe0490000e0b90009e0b900056
:101420006011b8009e0590000b38b100d501200076
:1014300082817100610164008703d1000683d300bb
:101440008984d3000884d3008502e900f8ff3a00bc
:10145000defd07000df0a70001f0a00065013700d8
:10146000f1ff2700f0ff2f006201370001f827008d
:1014700000002000f7ff37006000b800f5ff3700dc
:10148000dd0107000509780000000600809feb00e1
:10149000890107008f87e9000000e00000000600d6
:1014a0002800fa00889fbe008a9fbe008c9fbe0065
:1014b00007067800878669000c003b00030478006b
:1014c0008704780008f0a10009f0a100840f500003
:1014d000858f5800860f5900890f5c000300330088
:1014e0000cf0a20001003a000cf0a1002d01070051
:1014f0006400e1005f003200780147006408e10009
:10150000610032006c014700748557003200be0054
:101510001201be003a04be001a05be001e03900070
:10152000be0a90008503530006003d000004fd0044
:101530008104fd000205fd008305fd008703ea002c
:10154000050378000df8a3000400320060041400c5
:10155000e0841c0060051d00e0851d006022b800cd
:101560007d0320000d38e1008006eb000b00390000
:101570004433dd00f300b20083017300390037000b
:10158000848272000d027800e10664008b85d10030
:101590000a85d3008984d3000884d3008703e90037
:1015a000f7ff3b0008004000898048000a0149001d
:1015b0008b81490004003b0060001000e0801800af
:1015c00060011900e08119000358a30009003200ee
:1015d0008d82720084827200610260008301d100fa
:1015e0000281d3008180d3000080d3000603e8008d
:1015f0001b0037000348a30017003a000600e00074
:10160000170034000603e9000d00a30000004800a5
:101610008180480002014900838149000348a300fa
:101620000f003a000600e000090034000603e9005c
:101630000000400081804800020149008381490088
:1016400001003a000003eb000348a300f5ff32005d
:101650006022b80002003700848272006182660056
:10166000e900070003f0a1000cf0a70003f0a000c0
:10167000e0003700640147006408e10002003a001e
:101680000df8a300d8003a003200be001201be00df
:10169000d80037001400fa00889fbe008a9fbe0061
:1016a0008c9fbe000004be000205be00680047001b
:1016b0000a90be000890be00280107000070a70035
:1016c0000bf0a1000bf8a30020003a009e09900047
:1016d0000e099000fe0090006e0090009e029000a7
:1016e0003443200084825200c20032000a003c00d1
:1016f000b4fc2f000428e100140034008301d10061
:101700000281d3008180d3000080d3008502e800ed
:10171000faff3a00b7003700b40020000428e100c7
:1017200007003c00000040008180480002014900a1
:10173000838149008502e900faff3a00ad003700d5
:101740000300280002002000010037006011b800eb
:101750006000b800a70037002800fa00889fbe008c
:101760008a9fbe008c9fbe0003866b008d00070021
:101770006400e100440032006408e1004a003200e5
:101780006100e100460032006108e10049003200da
:10179000ec0647006000b8003d02be003d03be00fd
:1017a000f48657006011b8003d04be003d05be0040
:1017b0007d0320000b0037000000a0008d06e9002b
:1017c000130032000402420085824a0006034b00e7
:1017d00087834b00000040008180480002014900df
:1017e000838149000802520089825a000a035b0083
:1017f0008b835b00f0ff3b000802420089824a00b5
:101800000a034b008b834b008d06e900edff3a0085
:101810008482720086827200f707b20087827200ab
:1018200001003200150020001e0490003e0b9000c5
:1018300006035400e63fb0000368a300070032002f
:101840000000a7000500a0008301d1000281d300a1
:101850008180d3000080d3000603e8008301d1001b
:101860000281d3008180d3000080d3000002eb000e
:101870000482d2006400070003f0a1000cf0a7006e
:1018800003f0a0005b003700640247006408e10039
:10189000550032003400be003401be00f6ff3700b0
:1018a0006108e100500032006011b8006000b8002b
:1018b000f1ff370003ff270002002000fbff370085
:1018c000889fbe00830478000300e0002c003500f0
:1018d00003003c0000827000040271002600320008
:1018e00036432000c50020008383cf000a00390062
:1018f0000541b1008283cf00070039000541b100e6
:101900008183cf00040039000541b1008083cf00fe
:10191000010039000541b10085c353006022b800c1
:10192000120032000a003b008482720061026000f3
:101930008301d1000281d3008180d3000080d300d5
:101940000603e8008743e800f7ff3a000700370086
:101950000000400081804800020149008381490065
:101960000603e9008743e900f9ff3a002600070073
:1019700009f0a70003f0a0004f04be00000006001d
:1019800060001000e080180060011900e08119007b
:10199000d3ff3b00033e2c00f7ff370007f0a20007
:1019a000bffe3700680447000294be000094be00ea
:1019b000fc0447008694be008494be0009007800b1
:1019c00066000700080078006400070099007800ae
:1019d000814f70000b003b000800be009300070021
:1019e0004f00b10003003700f3ff2700f2ff2f0084
:1019f0006110b9004f06be004f05be004f04be0087
:101a00000080fa00000006001800200057002000a7
:101a1000080453000d003d000600200097fc2f0035
:101a20000740e1001e003400848272006102600001
:101a30008301d1000281d3008180d3000080d300d4
:101a40000804e800f8ff3a00470020006104600045
:101a500005047400040464000d00320061004000bd
:101a6000e080480060014900e081490003b8a5001a
:101a7000070032000603e8006538e10004003a0080
:101a80008301d1000281d3008180d3000080d30084
:101a9000f87f20000830e1000300350008037800db
:101aa0006000b8006011b8004433dd00f300b200fc
:101ab0008301730000000600889fbe008a9fbe005d
:101ac0008c9fbe000404be000605be00809fbe00c1
:101ad000829fbe0063000700040678000800be0075
:101ae0000a01be005f000700840678004f03be00b5
:101af0004f02be008d4f76007fb097001300330079
:101b0000f0ff2f008b8f6b0006003b000d06660078
:101b10000c00a7000a00370007f0a6001000200004
:101b20000a003700880f5200898f5a008a0f5b0025
:101b30008b8f5b00030039001000200001003e0085
:101b40000000200007f0a7000000ea004f06be00da
:101b50004f05be004f04be00000006008000780064
:101b60005002be005003be004439de00f700b20050
:101b7000f37f200003016100090032000218e10038
:101b800016003a008501720083017300838173009f
:101b90000008200015003a00400020001300370024
:101ba00085017200830173008381730005003a0090
:101bb00004a8be0006a8be00100020000b003700dd
:101bc0000201e9000402420085824a0006034b003c
:101bd00087834b000748a300f9ff32000740a000ad
:101be00004a8be0006a8be002000200080009800c7
:101bf00092009800000006000003be00defb070014
:101c00006220e100020032000600be00050005006f
:101c1000e507b100f107b20004f0230084807000f2
:101c200007f0a70001f0a00024000500e4824000b6
:101c30001078a30007003200640240001178a3006e
:101c40003400be001401be00040032000330a700bf
:101c5000000006003500be001501be000330a000e4
:101c60000000060005ff2700058261000700320022
:101c70000428e100010032002400050006000700ee
:101c800001003a00440005000408050002000700b6
:101c9000f9ff3a00140005006f82610081027000b4
:101ca00085027100850272000000060000017800c4
:101cb00000c2b300010037000201e8009240780042
:101cc00080cf5000fcff3200e9cf5000faff320015
:101cd000d0c2b30080cf500003003a000201e800f8
:101ce00014c0b300050037000042eb00b0c2b300df
:101cf00080cf500001003a000201e8008000eb00b4
:101d000005fd2f00040037006a08b900008041007b
:101d1000850040000201e8009201fb0005804100bf
:101d2000e90f5000f8ff36000404e0000100320023
:101d30008100ea0001007800000006008001eb004d
:101d400002003700817178008301e800828f510022
:101d5000fcff3a0000000600800078003004e0003c
:101d6000feff3a00010050000000e90000000600fc
:101d70008001780000017800314078000059780037
:101d80000004e000fcff3a000300780000000600b9
:101d90000003780080027800020278008001eb00e6
:101da000080037000402e90063c07800805a780018
:101db0008301e8000004e00002003a008000eb002c
:101dc00006003700828f5100f6ff3a00fbff370014
:101dd0000040eb0080f07a008100e800848f500022
:101de000fbff3a0006007800000006000c00fa0035
:101df000889fbe0000047800cfb09700f0ff270056
:101e0000d0bf9f008004eb0099bf9f0088bf9f0058
:101e1000a8bf9f00200c2000b0bf9f007881570012
:101e2000708057005f0007000fb8970009487800de
:101e30000fb8970008045000080078004f04be0057
:101e40000080fa0000000600889fbe008a1f78000c
:101e5000804078000004e00021003d008040ea005e
:101e6000d0c6b30080cf5000090034008104fb00cd
:101e700042062000110009008204d8000001780009
:101e8000010078004311dd006a1f21001f003700a8
:101e90000100fb00631f210039003700a200200071
:101ea000110009000200d80000017800010078004c
:101eb0004311dd00030141004300dd000300400049
:101ec0003002be002003be0042209000d2209000cd
:101ed000f221900062219000a0fc07002e00370044
:101ee000d0c6b30080cf5000230034008104fb0033
:101ef00042062000110009008204d8000001780089
:101f0000010078004311dd006a2a21000a01410026
:101f1000a8002000110009000800d8004300dd00df
:101f20000a00400040229000d022900060239000e0
:101f3000f02390000288900092889000b28990006f
:101f40002289900085fc0700801f7800010278003c
:101f5000110009008804d8000102fd004f0078003c
:101f60000402fb004322dd000a0242005403be00cb
:101f70004402be00d8ff37000100fb00632a2100a5
:101f8000eacf5000c5ff3c004300dd0003004000e5
:101f90005001be004000be004f0578004f04be0057
:101fa000000006008f03b000889fbe008a9fbe001d
:101fb0008c9fbe008e1f7800e0b79f00f1b79f0096
:101fc00082bf9f000000eb00a0b79f00e60437002f
:101fd0008001eb0050c2b30080cf500009003200f6
:101fe0000100fb00efb09700ec040700e10f400098
:101ff000dd043200afb097008100e800a1b79f0078
:10200000d90437007fb1970092407800d0c2b30066
:1020100080cf50000c00320007003c006d405000a3
:1020200080cf50000d0032006b40400080cf500048
:1020300019003a000e00370000c3b30080cf5000f3
:1020400015003a000f0037000330a0007fb2970060
:102050000402e800f4b79f00eaff37000300a00085
:10206000ffb297008502e800f5b79f00e5ff370053
:102070000310a0007fb697000c06e800fcb79f0095
:10208000e0ff37000320a0007fb097000000e800c9
:10209000f0b79f00dbff37000318a30001003200f8
:1020a0000300a1000338a300010032000320a100b7
:1020b0000100fb0002fd2f0002004000e90f50006c
:1020c00010003e008000eb00c1b79f0002027800c4
:1020d0004fb197006a10b900ffb297001501fb00dd
:1020e0000001410004014100c2b79f005500fb0000
:1020f000f5b79f0004004000e90f50000d003e00be
:10210000f3ff37000006eb00ccb79f00a0c2b3007e
:1021100080cf500007003a000fb89700c000780049
:1021200080bf9f00c1b79f007fb197000201e80008
:10213000f2b79f00e0c2b3007fb29700944f100047
:1021400021003a00830678000de0a0008400e8003a
:1021500064405000914f100004003200f1b79f001e
:102160008002eb00b5b79f00100037000fbe97004c
:102170004c0078008cbf9f00b0b79f00ffb0970065
:102180008180e800f1b79f00130037003fb297004d
:102190006a20b9000000410003004000b0b79f0072
:1021a000ffb297008502e800f5b79f007fb6970061
:1021b0001c01fb0003fd2f0003004100e90f50004c
:1021c000f2ff360004003700830678000dc0a0003f
:1021d0000000eb00b0b79f007fb19700b2407800dd
:1021e000f2b79f00c17f9f00c0c6b30080cf5000f0
:1021f0002700320014003c006840500080cf50009f
:102200009d00320009003c006c40500080cf50001f
:10221000290032006b40400080cf50007200320035
:102220000104e000560432008e00370060c6b3009f
:1022300080cf50001c0032006340400080cf50002f
:1022400088003a008c00370030c7b30080cf5000c0
:102250001c00320007003c006440500080cf50005a
:10226000130032000040e80080cf50007d003a00ab
:102270001100370050c7b30080cf50007d003200fe
:102280006340400080cf500076003a000b003700da
:10229000000028000d48a30001003a0000012000c2
:1022a00080867600ccff37000da0a00072003700ba
:1022b0000d60a000700037000d50a0000d70a00050
:1022c0006d0037008fb997004300780083bf9f00ef
:1022d000000478000000e00001003a00683f21009f
:1022e0008004eb00010037008104e80089007800d9
:1022f000088044001004e000fbff3a003fb2970062
:102300000400e00003003200890f52000100310098
:10231000840478000007eb00cfb29700898f520049
:1023200001003600098752004368de00e1066000c4
:1023300019003a000d06780009003700efb0970049
:102340000002200015040700e10f400003003200e6
:102350002fb097000000e800a0b79f000c06e8002f
:102360008e0f5600f5ff3a000087eb000a00370099
:10237000880078003100fb0001047800efb097007e
:1023800006040700e10f400003003200afb09700e1
:102390008100e800a1b79f000900e90080047800ef
:1023a000e10f4000f2ff3a000006eb000d00e000f4
:1023b0000a003a00ec033700efb09700000220005b
:1023c000f6030700e10f4000030032002fb1970031
:1023d0000201e800a2b79f000c06e8008e0f56002d
:1023e000f5ff3a00e00337008fb99700430078000b
:1023f00083bf9f00cf80de0001017800820178005a
:102400000205be000004be000203be000002be00c2
:102410004822de00482edd0004027600c47f9f00c3
:102420000d48a3000a0032000404e0000800320056
:10243000e14f420006003200d1fb2f00018047002f
:102440000448780018409800290020000200370056
:10245000d07f9f0019002000d2fb2f00028447008c
:10246000a6ff3700c3fb2f0003844700190020009c
:10247000a2ff37000d0cb300007020000082660040
:10248000270232000dc8a3000200320064002000c1
:10249000b4b79f000d48a300050032000fba9700a3
:1024a0004401be004400be0084bf9f00040037000a
:1024b0008fba97004500be0085bf9f009cfb0700b8
:1024c000e0af9f00f1af9f0082b79f0093b79f00de
:1024d0006022b8006033b8006fa89700ffa897008b
:1024e0000fb197009fb19700b0fb07000000e0001c
:1024f0000a003d006fa89700ffa897000fb1970052
:102500009fb1970003f0a200e0af9f00f1af9f00e2
:1025100082b79f0093b79f003d00b3000000eb001f
:1025200080a79f006022b8006033b8006fa89700b2
:10253000ffa897000fb197009fb19700a0fb07007d
:102540000000e000340032006fa89700ffa8970059
:102550000fb197009fb197009efb070003fc2f006f
:1025600003814700c6fb07000fa097000000e900a9
:102570006300b900a2002000110009000200d80089
:102580008000fd0081a79f000100e00002003d00e7
:102590000100e90080a79f000fa497000840ea000f
:1025a00029fe07006faa9700ffaa97000fb39700b4
:1025b0009fb39700e9fa0700a0af9f00b1af9f005b
:1025c000c2af9f00d3af9f006022b800060020007a
:1025d00007ff230075fb07000000e00002003d003c
:1025e0000800e9000b0037006022b8000600200058
:1025f000470224002fa89700bfa897004fa9970073
:10260000dfa99700a1fb07000000e00002003500f1
:102610000800e80080a79f003fb29700f80f520023
:1026200057003c00d0c6b300804f5200290036004e
:102630000485fb0042062000110009000285d80035
:1026400000017800010478004311dd006b1f2100b8
:102650000b0141006022b8000600200007fe2300a5
:102660000288900092889000b289900022899000a0
:10267000bafa0700a9002000809fbe0011000900df
:102680000984d800000478004f00be004344dd00f8
:102690000b04440048229000d82290006823900048
:1026a000f8239000adfa0700801f7800010278003f
:1026b000110009000985d8000102fd004f007800d3
:1026c0004322dd000b0242005403be004402be0060
:1026d0001f0037000480fb00691f2100ea4f5200f1
:1026e00014003600a2002000110009000280d8006a
:1026f00000017800010478004311dd000901410068
:102700006022b8000600200007fe2300422090004f
:10271000d2209000f2219000622190008ffa0700f1
:102720004344dd00090444003802be002803be0013
:10273000070037004300dd00090040006022b800b8
:102740000600200007fe23005001be004000be002e
:1027500082fa07000002be000203be006fa89700c5
:10276000ffa897000fb197009fb197004cfb07009f
:10277000e0af9f00f1af9f0082b79f0093b79f002b
:102780000fa49700e90f540015003c006022b80028
:102790006033b8006fa89700ffa897000fb19700ab
:1027a0009fb1970006fb07000000e00032003200f6
:1027b0006fa89700ffa897000fb197009fb19700ef
:1027c000b4fb0700e00f5000e08f5800e00f590005
:1027d000e08f590028003a00e10f54002600340031
:1027e0000400200005002e00b6e02200170124009e
:1027f0002fa89700bfa897004fa99700dfa99700bf
:10280000eafa07000000e00002003d0073005400f7
:10281000010037007200540080a79f000fc097008e
:1028200089fd0700a0af9f00b1af9f00c2af9f001e
:10283000d3af9f000002be000203be006fa8970046
:10284000ffa897000fb197009fb19700c2fb070048
:1028500090fb07000205be000004be006000b80047
:102860006011b800a0a79f00b1a79f00c2a79f005a
:10287000d3a79f002e0037006fa89700ffa89700ee
:102880000fb197009fb1970082fb07000205be00c1
:102890000004be00e00f5000e08f5800e00f590028
:1028a000e08f59000200350005fc070013003700d7
:1028b00010002000010020006011b8000800600036
:1028c000898060000a0161008b8161008b03d10067
:1028d0000a83d3008982d3000882d30000007200eb
:1028e000818072000201730083817300f4fb070092
:1028f0000002be000203be00e9fa07000002be00ab
:102900000203be006fa89700ffa897000fb19700c1
:102910009fb1970021fc0700a0a79f00b1a79f00cf
:10292000c2a79f00d3a79f000000eb0080a79f00d5
:1029300014c0b300653521000b0037000400fb0014
:102940004300dd00050040005001be004000be0015
:102950000040e10001c8e10002d0e10003d8e1003d
:10296000030039000442e800f44f5200f3ff3a003c
:10297000c47f9f000400fb00bfb0970000804000b0
:102980008fa09700010040004fb197000007510051
:10299000bfb197000300e000010032000e07e9001c
:1029a00063806600010032000e07e9000d28a300d5
:1029b00026003200e18066000d18a3000c003200f2
:1029c000d00220000100e00001003a000080e90090
:1029d000efb0970071020700e10f400018003200cd
:1029e0002fb297000402e800a4b79f00140037003c
:1029f0000100e00012003200efb09700000220005a
:102a000066020700e10f40000d003200afb29700f0
:102a10008502e800a5b79f0009003700efb09700d6
:102a2000000320005d020700e10f400003003200b8
:102a30002fb697000c06e800acb79f000e07e90020
:102a40000e00e000f5ff3c003d0037000d38a3000c
:102a50000a0032000b003700efb0970000022000a0
:102a60004e020700e10f4000030032002fb0970034
:102a70000000e800a0b79f000e07e9000e00e0008c
:102a8000f5ff3c00e18066000d18a3000c00320049
:102a9000d00220000100e00001003a000080e900bf
:102aa000efb097003d020700e10f40002400320024
:102ab000afb097008100e800a1b79f002000370069
:102ac0000100e0001e003200efb09700000220007d
:102ad00032020700e10f4000190032002fb19700c9
:102ae0000201e800a2b79f00150037000000fb00bc
:102af0004300dd0061352100010040003002be00ce
:102b00002003be000800be000a01be0002f9070053
:102b1000a4002000050020006033b80005f907007c
:102b20000003b000efb097001c020700e10f400067
:102b300003003200afb197008301e800a3b79f0004
:102b40004f7a97000440e900c07f9f00e14f4000aa
:102b5000e6ff3a000b003700efb0970000032000bb
:102b60000e020700e10f400003003200afb29700f1
:102b70008502e800a5b79f000fa097000000e900bc
:102b800080a79f000fa097000000e000f2ff3c002c
:102b90003fb6970020c1b300f20f560001003c0081
:102ba0006fe09700c07f9f00cf7897000100fb0087
:102bb0003fb1970000005100e0a79f000104e00032
:102bc00008003200efb09700e0022000f301070098
:102bd000e10f400003003200afb197008301e8002d
:102be000a3b79f004f78970097fc07000002be0034
:102bf0000203be002fa09700bfa097004fa197002f
:102c0000dfa1970055f90700a2fa07001e00370060
:102c10000000fb004300dd006c3521000c0040008b
:102c20003002be002003be000800be000a01be0044
:102c3000b9f80700a4002000050020006033b800a8
:102c4000bcf807000003b000efb09700d301070005
:102c5000e10f4000030032002fb297000402e800a9
:102c6000a4b79f00cf7a97000500fb004300dd006a
:102c70000c0040003002be002003be000800be0071
:102c80000a01be00abf807000205be000004be004a
:102c90004f7e97000c40e900c07f9f00e14f40004d
:102ca000dbff3a000006eb0009003700efb09700a9
:102cb00000032000b9010700e10f400003003200cb
:102cc0002fb097000000e800a0b79f000c06e800b6
:102cd000efa09700810f5600f4ff3a000d38a300d3
:102ce000a10132000e00e0009f0134000006eb005d
:102cf000efb0970000022000a8010700e10f40009c
:102d0000030032002fb197000201e800a2b79f0034
:102d10000c06e8008e0f560093013200f4ff3700d6
:102d20000d007800000cb20028003a000d00e00011
:102d300005003d008fb997004305be004304be0067
:102d400083bf9f00140037000d48a3000b00320022
:102d50000fba97004400be0084bf9f004f89de0079
:102d6000cf91de000002be000203780082037800eb
:102d70000605be000404be00070037008fba9700a6
:102d80004500780085bf9f0000047800cfc4de00b6
:102d9000090578008a057800e00f5400e08f5c0098
:102da000e00f5d00e08f5d0020003d003d00b300be
:102db0006000b8006011b800080450008984580011
:102dc0000a0559008b855900180037000d00e000f6
:102dd00005003d000fbe97004c05be004c04be0030
:102de0008cbf9f00110037000d48a300080032007f
:102df0008fba97004500be0085bf9f000401780090
:102e0000840178000205be000004be000700370000
:102e10000fbe97004c0078008cbf9f000004780024
:102e2000090020000a0020000b0020003fb097009e
:102e30000000e00007003a00e00f5400e08f5c0063
:102e4000e00f5d00e08f5d0002003a0011002000fd
:102e5000b1b79f000d0778000e0cb20000042000ef
:102e6000800f57002f00320003003c000e00e000ee
:102e7000070032003f00370000082000800f570095
:102e800014003200000c2000800f570039003a0077
:102e900014c0b300653521000b0037000400fb00af
:102ea0004300dd00050040005001be004000be00b0
:102eb0000040e10001c8e10002d0e10003d8e100d8
:102ec0002b0039000442e800f44f5200f3ff3a00af
:102ed0002700370000012000010020006011b80029
:102ee00014c0b3000040e10001c8e10002d0e100dd
:102ef00003d8e1001e003900450020000000d0008a
:102f00008180d2000281d2008381d2008502e90053
:102f1000faff3a000442e800f04f5200f1ff3a0095
:102f20001300370080002000010020006011b8006d
:102f300014c0b3000040e10001c8e10002d0e1008c
:102f400003d8e1000a0039003c0020000000d00056
:102f50008180d2000281d2008381d2000c06e90078
:102f6000faff3a000442e800f54f5200f1ff3a0040
:102f7000c47f9f00cf7897000100fb003fb197000e
:102f8000820f500002003d00c27f9f000400370006
:102f9000bfb19700808f510001003d00b0b79f0086
:102fa0004fb297000400e000040032006380660026
:102fb000020032000402e900c4b79f000de8a3003c
:102fc0000b003200cfb297003fb697008c8f5200b3
:102fd00003003c000000eb00c0b79f000400370076
:102fe000cfb097003fb1970082805000c1b79f00db
:102ff000cf7997000300fb000002eb0094a79f002d
:10300000cfb29700808f520002003400008052003f
:1030100090a79f000d28a30037003200e1806600d2
:103020000d18a3000c003200d00220000100e000c7
:1030300001003a000080e900efb09700d7000700d8
:10304000e10f40000e0032002fb697000c06e8009a
:10305000acb79f000a0037000100e0000800320012
:10306000efb0970000022000cc000700e10f400005
:10307000030032002fb097000000e800a0b79f00c7
:103080009fa097000100e0000f0032000006eb0057
:10309000efb0970000032000c0000700e10f4000e0
:1030a000030032002fb197000201e800a2b79f0091
:1030b0000c06e8009fa19700830f5600f4ff3a002a
:1030c0000002eb0094a79f00bfb29700c328dd0069
:1030d000e03421008080400091af9f004228dd0055
:1030e0006400500080af9f006328b900f0a79f00e4
:1030f00063065000820037001fa697000c00e00016
:1031000011003200688066000f003a000006780067
:10311000efb0970000022000a0000700e10f400080
:10312000030032002fb097000000e800a0b79f0016
:103130000c06e8009fa09700810f5600f4ff3a00ac
:103140000001eb0092a79f00e18066000d18a3002c
:103150000c003200d00220000100e00001003a0023
:103160000080e900efb097008c000700e10f4000fd
:10317000d5ff3200afb197008301e800a3b79f00ed
:10318000d1ff37000100e000cfff3200efb0970021
:103190000002200081000700e10f4000caff32005a
:1031a0002fb297000402e800a4b79f00c6ff3700c3
:1031b00000042000800f57003000320003003c0064
:1031c0000e00e000070032003d003700000820003c
:1031d000800f570011003200000c2000800f5700b4
:1031e00037003a001fa897003002be002003be003f
:1031f0000800be000a01be0047f70700a400200037
:10320000050020006033b8004af7070004c3b3008c
:1032100004424000c47f9f0029003700d53f2100b1
:10322000d5b79f000d58a30002003a00e0402100ee
:10323000d0b79f0014002000050020006033b800c4
:103240008fa897008100e900050033000402d00038
:103250008582d2000683d2008783d200f9ff37002f
:103260000800be000a01be002bf707006f006000d7
:103270005fb1970062407800100037001400200012
:10328000050020006033b8008c0178008301e9005c
:10329000050033000402d0008582d2000683d200ec
:1032a0008783d200f9ff37000800be000a01be0084
:1032b00019f70700674060000043b000c07f9f001f
:1032c0004f7a97000400fb00efb09700330007002f
:1032d000e10f400003003200afb297008502e80022
:1032e000a5b79f001fa897006800500090af9f00ef
:1032f0008fa89700e480500081af9f0063065600be
:10330000d0ff2f003fb197000090b900ffa19700b8
:103310000080410063005000800f5600a4ff3a0077
:103320000d38a300100032001fa297000400e00037
:103330000d0034000006eb00efb097000002200003
:1033400016000700e10f400003003200afb2970003
:103350008502e800a5b79f000c06e8001fa09700b3
:10336000800f5600f4ff3a007fb19700b24078001a
:10337000f2b79f00c17f9f000104e00014fb3a00f8
:103380002fb097004f0778004f06be004f05be00d4
:103390004f04be008f03b10000000600889fbe00ee
:1033a0000001780001047800b10090000118a3002a
:1033b0003d0032000198a30003003a00180090007d
:1033c0000000e00038003a000190a00031049800ad
:1033d00082047800f90fb200180090000000e000ad
:1033e00002003a0028009000000c7800ea8f540098
:1033f00006003a00380090000078a30003003a006d
:1034000088007800d0002000e4ff070098009000ba
:1034100058009000808f50000b0032000100e8003f
:10342000100498001800780009587800000c780003
:1034300011c0b300a044210001487800ea8f540075
:103440000600320019003700880078000940780033
:10345000190007008004780014003700380090003d
:103460000088a3001100320018019000a80090000d
:103470004800900067f4070098009000810f50000a
:1034800004003200380090000003b30030049800bc
:103490008084eb000000eb001004980028009000ee
:1034a000000c7800010037008084eb0009007800f0
:1034b0004f04be00000006000200fa00889fbe0014
:1034c000a0ff9f0001047800b10090008104780003
:1034d0000904b200020032000000fb003600370091
:1034e0000118a30005003a000103b300310498005d
:1034f000190498000080eb002f003700580090005e
:103500000000e00006003a00480090001200200091
:10351000e68057003ff407001904980024003700a4
:10352000280090000000e00008003a0060442100fc
:1035300020049800000c780020002000500498001f
:10354000100498000130a000310498001801900088
:10355000a8009000480090002ef40700280090007a
:10356000000c78000080eb00100498001800780030
:10357000aff8970001587800000c78002ff89700fa
:10358000ea4f50000a003a00380090000088a3007b
:103590000700320018019000a80090004800900039
:1035a0001cf4070019049800a8009000010c780092
:1035b000aff897000100fb004f04be000080fa0046
:0435c0000000060001
:020000040000fa
:020000040005f5
:0457f400021e000091
:020000040000fa
:020000040005f5
:0457f800bdfa0000f6
:020000040000fa
:020000040005f5
:0457fc007f3e0000ec
:020000040000fa
:10000800dc020000dc020000dc020000dc02000070
:10001800dc020000dc020000dc020000dc02000060
:10002800dc020000dc020000dc020000dc02000050
:10003800dc020000dc020000dc020000be4200001e
:10004800dc020000dc02000086370000403b0000b4
:10005800283b0000dc020000dc020000dc0200009b
:10006800dc020000dc020000dc020000dc02000010
:10007800dc020000dc020000dc020000dc02000000
:10008800dc020000dc020000dc020000dc020000f0
:10009800dc020000dc020000dc020000dc020000e0
:1000a800dc020000dc020000dc020000dc020000d0
:1000b800dc020000dc020000dc020000dc020000c0
:1000c800dc020000dc020000dc020000dc020000b0
:1000d800dc020000dc020000dc020000dc020000a0
:1000e800dc020000dc020000dc020000dc02000090
:1000f800dc020000dc020000dc020000dc02000080
:10010800dc020000dc020000dc020000dc0200006f
:10011800dc020000dc020000dc020000dc0200005f
:10012800dc020000dc020000dc020000dc0200004f
:10013800dc020000dc020000dc020000dc0200003f
:10014800dc020000dc020000dc020000dc0200002f
:10015800dc020000dc020000dc020000dc0200001f
:10016800dc020000dc020000dc020000dc0200000f
:10017800dc020000dc020000dc020000dc020000ff
:10018800dc020000dc020000dc020000dc020000ef
:10019800dc020000dc020000dc020000dc020000df
:1001a800dc020000dc020000dc020000dc020000cf
:1001b800dc020000dc020000dc020000dc020000bf
:1001c800dc020000dc020000dc020000dc020000af
:1001d800dc020000dc020000dc020000dc0200009f
:1001e800dc020000dc020000dc020000dc0200008f
:0801f800dc020000dc02000043
:020000040000fa
:10020800dc020000dc020000dc020000dc0200006e
:10021800dc020000dc020000dc020000dc0200005e
:10022800dc020000dc020000dc020000dc0200004e
:10023800dc020000dc020000dc020000be4200001c
:10024800dc020000dc02000086370000403b0000b2
:10025800283b0000dc020000dc020000dc02000099
:10026800dc020000dc020000dc020000dc0200000e
:10027800dc020000dc020000dc020000dc020000fe
:10028800dc020000dc020000dc020000dc020000ee
:10029800dc020000dc020000dc020000dc020000de
:1002a800dc020000dc020000dc020000dc020000ce
:1002b800dc020000dc020000dc020000dc020000be
:1002c800dc020000dc020000dc020000dc020000ae
:1002d800dc020000dc020000dc020000dc0200009e
:1002e800dc020000dc020000dc020000dc0200008e
:1002f800dc020000dc020000dc020000dc0200007e
:10030800dc020000dc020000dc020000dc0200006d
:10031800dc020000dc020000dc020000dc0200005d
:10032800dc020000dc020000dc020000dc0200004d
:10033800dc020000dc020000dc020000dc0200003d
:10034800dc020000dc020000dc020000dc0200002d
:10035800dc020000dc020000dc020000dc0200001d
:10036800dc020000dc020000dc020000dc0200000d
:10037800dc020000dc020000dc020000dc020000fd
:10038800dc020000dc020000dc020000dc020000ed
:10039800dc020000dc020000dc020000dc020000dd
:1003a800dc020000dc020000dc020000dc020000cd
:1003b800dc020000dc020000dc020000dc020000bd
:1003c800dc020000dc020000dc020000dc020000ad
:1003d800dc020000dc020000dc020000dc0200009d
:1003e800dc020000dc020000dc020000dc0200008d
:0803f800dc020000dc02000041
:020000040000fa
:1035c4004d4500004f5700000d0a0000006900003f
:1035d4006e310000203d000020250000642c000016
:1035e400206900006e320000203d0000202500000c
:1035f400642c0000206900006e330000203d0000b0
:1036040020250000640d00000a000000424900006b
:1036140054200000256400002049000053200000cd
:10362400484900000d0a000000420000495400000f
:10363400202500006420000049530000204c0000b5
:103644004f0d00000a000000535000004920000004
:103654004952000051200000434f0000554e000025
:10366400542000003d200000257500000d0a0000d4
:103674000053000050490000204300004d44000066
:10368400204300004f5500004e540000203d000030
:1036940020250000750d00000a00000053500000b2
:1036a40049200000494e0000464f0000204300001e
:1036b4004f5500004e540000203d0000202500001e
:1036c400750d00000a00000053500000492000005e
:1036d4005245000041440000204300004f550000c3
:1036e4004e540000203d000020250000750d000010
:1036f4000a00000053500000492000005752000007
:103704004954000045200000434f0000554e00007e
:10371400542000003d200000257500000d0a000023
:103724000053000050490000204f0000564500009f
:10373400524600004c4f0000572000004249000050
:1037440054200000203d0000203100000d0a00003c
:103754000053000050490000204f0000564500006f
:10376400524600004c4f0000572000004249000020
:1037740054200000203d0000203000000d0a00000d
:103784000053000050490000315300005441000030
:10379400542000003d200000307800002530000057
:1037a400345800000d0a0000005f00005350000070
:1037b4004931000049460000203d0000203100004e
:1037c4000d0a0000005f0000535000004931000062
:1037d40049460000203d0000203000000d0a000092
:1037e400005f0000535000004931000049450000cb
:1037f400203d0000203100000d0a0000005f0000a1
:10380400535000004931000049450000203d0000ac
:10381400203000000d0a0000000d00000a520000d4
:1038240065740000757200006e650000642000007d
:10383400566100006c750000652000003d2000000a
:10384400256600000d0a0000006100006e610000a2
:103854006c6f000067310000203d0000202500004f
:10386400640d00000a000000616e0000616c00003d
:103874006f670000322000003d2000002564000036
:103884000d0a0000006100006e6100006c6f000012
:1038940067330000203d000020250000640d000077
:1038a4000a000000616e0000616c00006f67000098
:1038b400342000003d200000256400000d0a0000b3
:1038c400006100006e6100006c6f0000673500004d
:1038d400203d000020250000640d00000a000000c7
:1038e400616e0000616c00006f670000362000000c
:1038f4003d200000256400000d0a00000054000073
:10390400656d000070200000536500006e730000b8
:103914006f720000205b00004a3600005d2000004a
:103924006973000020250000642000006465000025
:103934006772000065650000730d00000a00000056
:10394400546500006d70000020530000656e000097
:10395400736f0000722000005b4a0000375d0000b6
:10396400206900007320000025640000206400002a
:103974006567000072650000657300000d0a0000b1
:1039840000540000656d00007020000053650000c5
:103994006e7300006f720000205b00004a38000064
:1039a4005d200000697300002025000064200000f1
:1039b400646500006772000065650000730d000017
:1039c4000a000000546500006d70000020530000e0
:1039d400656e0000736f0000722000005b4a0000f7
:1039e400395d000020690000732000002564000098
:1039f40020640000656700007265000065730000c4
:103a04000d0a000000540000656d000070200000e5
:103a1400536500006e7300006f720000205b0000ad
:103a24004a310000335d000020690000732000006b
:103a340025640000206400006567000072650000d2
:103a4400657300000d0a000000540000656d00005d
:103a540070200000536500006e7300006f72000058
:103a6400205b00004a310000355d00002069000041
:103a740073200000256400002064000065670000d6
:103a840072650000657300000d0a00000054000018
:103a9400656d000070200000536500006e73000027
:103aa4006f720000205b00004a310000365d0000a8
:103ab40020690000732000002564000020640000d9
:103ac4006567000072650000657300000d0a000060
:103ad40000540000656d0000702000005365000074
:103ae4006e7300006f720000205b00004a3100001a
:103af400375d000020690000732000002564000089
:103b040020640000656700007265000065730000b2
:103b14000d0a000000250000752500007525000031
:103b240075250000750d00000a00000061630000a7
:103b34007453000065740000537400007562000043
:103b4400436d000064280000292000003d2000008f
:103b5400256400000d0a00000000000000000000c1
:103b64000000000000000000000000000000000051
:103b74000000000000000000000000000000000041
:103b84000000000000000000000000000000000031
:103b94000000000000000000000000000000000021
:103dd400000000000000000000000000202000009f
:103de400202000002000000047450000540000008f
:103df4005345000054000000434c000045410000be
:103e0400527c0000434c0000520000005245000068
:103e14005345000054000000484500004c4c00008d
:103e24004f2000004b49000054540000590000008a
:103e34005350000049320000544500005354000020
:103e440000000000f69e000048210000fa9e0000d9
:103e540058210000fe9e000068210000089f000019
:103e6400782100000e9f0000842100001a9f0000aa
:103e740096210000239f0000000000004341000041
:103e840052440000204900004e4600004f0000004c
:103e940053500000492000005354000041540000d6
:103ea40053000000444900004e000000444f00004d
:103eb4005554000000410000444300000054000039
:103ec400454d000050000000414400004342000002
:103ed4005553000059000000434f00004d500000ae
:103ee4004153000053000000409f0000e621000001
:103ef4004a9f00006c220000549f0000f42100003f
:103f0400589f0000302200005d9f0000ae24000096
:103f1400619f00006c260000669f0000cc27000013
:103f24006e9f000044230000239f00000000000057
:103f340053540000554200000043000053000000a9
:103f44009a9f00000e280000589f000032280000ad
:103f54009f9f000048280000239f000000000000ed
:103f64004a9f00005c280000589f0000722800004f
:103f7400239f000000000000485500004d30000061
:103f840031000000485500004d30000032000000b0
:103f9400485500004d300000330000004855000033
:103fa4004d3000003400000046490000424f00003c
:103fb40000540000454d0000503000003100000066
:103fc400544500004d500000303200000054000001
:103fd400454d0000503000003300000054450000ff
:103fe4004d5000003034000000540000454d0000e6
:103ff4005030000035000000544500004d500000d2
:104004003036000000540000454d000050300000e0
:1040140037000000544500004d50000030380000c7
:1040240000480000323000005f310000004800000a
:10403400323000005f3200000048000032300000df
:104044005f33000000480000323000005f3400009d
:1040540000000000be9f0000c49f0000ca9f000033
:10406400d09f0000d69f0000db9f0000e29f00006d
:10407400e99f0000f09f0000f79f0000fe9f0000f2
:1040840005a000000ca0000013a0000019a000006f
:104094001fa0000025a00000000000004c560000f6
:1040a4004c530000004900004e54000045530000ea
:1040b40054000000313600003a320000353a000066
:1040c40035360000004a0000756c00002020000016
:1040d400332000003230000031320000000d0000b7
:1040e4000a4600004f4300004520000043480000fa
:1040f4004153000053490000532000004c4f00007e
:1041040057200000564f00004c5400004147000067
:10411400452000004c4f00004144000020530000a3
:104124005749000054430000484500005220000055
:10413400424f00004152000044200000427500003c
:10414400696c0000742000006f6e000020250000e0
:10415400732000006174000020250000730d00002e
:104164000a00000043610000726400002054000053
:1041740079700000653a000020250000640d0000fd
:104184000a0000004361000072640000204e000039
:10419400616d0000653a000020250000730d0000e9
:1041a4000a000000566100007269000061620000ac
:1041b4006c650000204e0000616d00006573000016
:1041c4003a0d00000a000000286900006e7000002b
:1041d40075740000290d00000a000000286f00001b
:1041e4007574000070750000742900000d0a000049
:1041f40000280000696e00006f750000742900003b
:104204000d0a0000000d00000a000000000000007c
:10421400000000000000000000000000000000009a
:10422400000000000000000000000000000000008a
:10423400000000000000000000000000000000007a
:10424400000000000000000000000000000000006a
:10425400000000000000000000000000000000005a
:104264000000000000000000000000002009000021
:104274000020000000300000313200003334000020
:0c4284003536000037380000390000001b
:020000040000fa
:104290000200fa00000f78005200200061f72900a8
:1042a0001e007800ae0f07000080fa000000060034
:1042b0000200fa00000f78005200200021fa2900c5
:1042c0001e007800a60f07000080fa00000006001c
:1042d0000200fa00000f78005200200021fb2900a4
:1042e0001e0078009e0f07000080fa000000060004
:1042f0000200fa00000f78000000fe000000eb0052
:104300000080fa00000006000200fa00000f7800aa
:10431000c0d6200021ae29000600090031587800df
:104320000000eb000080fa00000006000800fa0020
:10433000300798000040eb00404798000040eb0039
:10434000304798000040eb00204798008000200094
:104350006f03070070c8b300f312070000000000ed
:104360000040eb00f0120700404798000040eb00cf
:10437000ed120700304798000040eb00ea120700fa
:10438000204798002e4090008080fb003e40900027
:104390000081fb004e4090000080fb00811f7800f0
:1043a000821f7800801f780090ae2900801f78005f
:1043b00000ab20008df60700e887570001ab200016
:1043c00010002000160c0700e0ff37000200fa0082
:1043d000000f7800e0e62000b71007000000eb00b7
:1043e0000080fa00000006000400fa0010079800a0
:1043f0001e0090002df60700000f78001e007800c8
:104400006d0707000000e000080032001e00780081
:10441000801f780080b02900801f7800c0d620005f
:1044200072f60700e4875700070037001e00780087
:10443000801f780070b12900801f7800c0d620004e
:104440006af60700e4875700c1d62000100020005c
:10445000f30b07000000eb000080fa0000000600ec
:104460000400fa00100798001e0090000ff60700e5
:10447000000f78001e007800740607000000e000be
:10448000080032001e007800801f780080b02900ec
:10449000801f7800c0d6200054f60700e48757003c
:1044a000070037001e007800801f780070b12900d7
:1044b000801f7800c0d620004cf60700e487570024
:1044c000c1d6200010002000d50b07000000eb0033
:1044d0000080fa00000006000400fa0010079800af
:1044e000220a0700000f78001e007800801f780065
:1044f00060b22900801f780000ab20003bf6070067
:10450000e487570001ab200010002000c40b070017
:104510001a0a0700000f78001e007800801f78003c
:10452000b0b32900801f780000ab20002ff60700f1
:10453000e487570001ab200010002000b80b0700f3
:10454000120a0700000f78001e007800801f780014
:1045500000b52900801f780000ab200023f607007b
:10456000e487570001ab200010002000ac0b0700cf
:104570000a0a0700000f78001e007800801f7800ec
:1045800060b62900801f780000ab200017f60700f6
:10459000e487570001ab200010002000a00b0700ab
:1045a000020a0700000f78001e007800801f7800c4
:1045b000c0b72900801f780000ab20000bf6070071
:1045c000e487570001ab200010002000940b070087
:1045d00040c2bf000044b2000004e000040032000a
:1045e00031b92900100020008d0b070003003700af
:1045f000b1ba290010002000890b070000128000ca
:10460000801f780030bc2900801f780000ab20009c
:10461000f6f50700e487570001ab200010002000ea
:104620007f0b070085c0bf00644060000004e0000d
:104630000400320071bd290010002000780b070033
:104640000300370051be290010002000740b070042
:1046500095c0bf00644060000004e0000400320028
:1046600031bf2900100020006d0b07000300370048
:1046700011c0290010002000690b07000000eb00aa
:104680000080fa00000006001800fa00200f9800d1
:104690002e08900085f50700100f98000000eb0031
:1046a000000f98006000b80060079800710798003c
:1046b0000000eb00500798000000eb004007980056
:1046c0000000eb00300798000000eb002007980086
:1046d0000000eb00100798000000eb00000f7800ce
:1046e0001e089000300f9800be089000e18f500027
:1046f000110032003e089000e10f500004003c0021
:10470000be0890000100e0000800320012003700ef
:104710003e089000e20f50000a003200be089000f0
:10472000e38f50000a0032000b00370060092000c0
:10473000000f980008003700600d2000000f98005f
:1047400005003700600a2000000f980002003700c3
:10475000600e2000000f980060c2a800000000005a
:10476000900020006a0207000e089000ee1107007a
:10477000000000000040eb00eb110700500798001c
:104780000040eb00e8110700400798000040eb00f4
:10479000e511070030079800300620005c02070092
:1047a0005e009000200798002e0090004800dd0079
:1047b00020079800ce009000f00f2000808060005d
:1047c0002e00900001007000200798002e0090003d
:1047d00000004000200798003e0090004700de00e7
:1047e000300798000000eb00100798001e009000b2
:1047f0004800dd0010079800be009000f00f200078
:10480000808060001e00900001007000100798007a
:10481000ae0090001e009000008f7000220020006b
:104820009e0078001e089000b00c070060079800fa
:10483000710798006e009000fe009000809fbe00ff
:10484000f0c02900801f7800c0d6200067f507005f
:10485000e6875700c1d6200010002000f00a0700ac
:10486000de009000811f780070c22900801f780050
:10487000c0d620005df50700e4875700c1d62000b0
:1048800010002000e60a07004e009000801f78000c
:1048900060c32900801f7800c0d6200053f50700b0
:1048a000e4875700c1d6200010002000dc0a070072
:1048b000be009000811f780050c42900801f78003e
:1048c000c0d6200049f50700e4875700c1d6200074
:1048d00010002000d20a07002e009000801f7800f0
:1048e00040c52900801f7800c0d620003ff5070092
:1048f000e4875700c1d6200010002000c80a070036
:104900009e009000811f780030c62900801f78002b
:10491000c0d6200035f50700e4875700c1d6200037
:1049200010002000be0a07001e007800801f7800db
:1049300020c72900801f7800c0d620002bf5070073
:10494000e4875700c1d6200010002000b40a0700f9
:104950000000eb000080fa00000006001c00fa00d6
:10496000300f98003e089000d0f40700200f980008
:104970000000eb00100f98000000eb00000f980003
:104980000000eb00700798000000eb006007980043
:104990000000eb00500798000000eb004007980073
:1049a0000000eb00300798006000b8001007980086
:1049b000210798000000eb00000f78002e089000ff
:1049c000e80f500003003c0080002000000f78003a
:1049d0000200370090002000000f78002e089000a1
:1049e0006101b900420f9800530f9800b0002000f9
:1049f000010020004e099000de099000800f510058
:104a0000818f590032003e004e089000de08900071
:104a1000006001000b0037000d0037000f00370069
:104a2000110037001300370015003700170037005a
:104a3000190037001b0037001d0037001f0037002a
:104a40002100370060082000300798002000370060
:104a5000600c2000300798001d003700600920001e
:104a6000300798001a003700600d200030079800ca
:104a700017003700600a2000300798001400370044
:104a8000600e20003007980011003700600b2000f6
:104a9000300798000e003700600f200030079800a4
:104aa0000b0037006009200030079800080037002d
:104ab000600a2000300798000500370060052000dc
:104ac0003007980002003700600d20003007980082
:104ad0001e0078008e01070060c2a80000000000e0
:104ae0003e00900010110700000000000040eb00a5
:104af0000d110700100f98000040eb000a1107008d
:104b0000000f98000040eb000711070070079800a5
:104b1000300620007e0107009e0890006107980083
:104b20006e0090004800dd00600798008e0890003d
:104b3000f00f2000808060006e0090000100700087
:104b4000600798006e009000000040006007980029
:104b50007e0090004700de00700798000000eb0028
:104b6000500798005e0090004800dd005007980054
:104b7000fe009000f00f2000808060005e0090003a
:104b80000100700050079800ee0090005e00900059
:104b9000008070004007980022002000ce009000a6
:104ba0002e089000d10b07001007980021079800ed
:104bb0001e019000ae019000829fbe00f0c029004f
:104bc000801f7800c0d6200088f40700e6875700d1
:104bd000c1d6200010002000110a07009e09900095
:104be000831f780070c22900801f7800c0d6200083
:104bf0007ef40700e4875700c1d620001000200093
:104c0000070a07000e089000801f780060c3290083
:104c1000801f7800c0d6200074f40700e487570096
:104c2000c1d6200010002000fd090700fe00900002
:104c3000811f780050c42900801f7800c0d6200052
:104c40006af40700e4875700c1d620001000200056
:104c5000f30907006e019000821f780040c529000b
:104c6000801f7800c0d6200060f40700e48757005a
:104c7000c1d6200010002000e9090700de019000e5
:104c8000831f780030c62900801f7800c0d620001e
:104c900056f40700e4875700c1d62000100020001a
:104ca000df0907004e009000801f780020c7290010
:104cb000801f7800c0d620004cf40700e48757001e
:104cc000c1d6200010002000d50907000000eb002d
:104cd0000080fa00000006000800fa002007980093
:104ce0002e009000f1f30700100798000000eb0081
:104cf000000f78001e009000300798003e009000e2
:104d0000e30f50004d0032003e009000e30f5000d2
:104d10000a003c003e009000e10f500025003200e8
:104d20003e009000e10f500033003c003e00900038
:104d30000000e0000e003200940037003e009000ba
:104d4000e50f50005f0032003e009000e50f50007c
:104d50004b0035003e009000e60f50006a00320024
:104d60003e009000e70f50007800320087003700c7
:104d700002002c00934724000000eb00e70207002c
:104d80005bee0700000f78001e007800801f78009f
:104d900010c82900801f7800c0d6200013f4070037
:104da000e4875700c1d62000100020009c090700ae
:104db0007600370002002c009347240010002000ea
:104dc000d60207004aee0700000f78001e007800a8
:104dd000801f780020ca2900801f7800c0d62000dc
:104de00002f40700e4875700c1d62000100020001d
:104df0008b0907006500370002002c009347240050
:104e000020002000c502070039ee0700000f7800df
:104e10001e007800801f780030cc2900801f7800a9
:104e2000c0d62000f1f30700e4875700c1d6200068
:104e3000100020007a0907005400370002002c00ff
:104e40009347240030002000b402070028ee07003a
:104e5000000f78001e007800801f780040ce2900e7
:104e6000801f7800c0d62000e0f30700e4875700d9
:104e7000c1d6200010002000690907004300370058
:104e800002002c009347240040002000a3020700ea
:104e900017ee0700000f78001e007800801f7800d2
:104ea00050d02900801f7800c0d62000cff3070023
:104eb000e4875700c1d620001000200058090700e1
:104ec0003200370002002c009347240050002000dd
:104ed0009202070006ee0700000f78001e0078001f
:104ee000801f780070d22900801f7800c0d6200073
:104ef000bef30700e4875700c1d620001000200051
:104f0000470907002100370002002c0093472400c6
:104f10006000200081020700f5ed0700000f780017
:104f20001e007800801f780090d42900801f780030
:104f3000c0d62000adf30700e4875700c1d620009b
:104f400010002000360907001000370002002c0076
:104f5000934724007000200070020700e4ed070072
:104f6000000f78001e007800801f7800b0d629005e
:104f7000801f7800c0d620009cf30700e48757000c
:104f8000c1d6200010002000250907000000eb001a
:104f90000080fa00000006000a00fa0040079800ae
:104fa0000000eb0084040700000f780010002000d0
:104fb0008104070010079800200020007e040700ed
:104fc00020079800300020007b040700300798007d
:104fd0003e009000ae0090001e0190009e017800ff
:104fe000801f7800811f7800821f7800831f78005f
:104ff000d0d82900801f780000ab20007bf3070089
:10500000ea87570001ab20001000200004090700c8
:105010000000eb000080fa00000006000400fa0027
:10502000100798001e00900020f30700000f780082
:105030001e007800801f780080d92900801f78002a
:10504000c0d6200069f30700e487570001ab2000b9
:1050500010002000f20807000000eb000080fa00ba
:10506000000006000400fa00100798001e009000df
:105070000ef30700000f7800110020001e007800da
:10508000790207000000eb000080fa000000060033
:105090000400fa00100798001e00900003f30700b8
:1050a000000f78001e007800190007000000eb00d8
:1050b0000080fa00000006000200fa00000f7800ed
:1050c00042070700460707004a0707004e07070088
:1050d0005207070040c2a9000000eb000080fa0060
:1050e000000006000400fa00100798001e0090005f
:1050f000eef20700000f78008000eb001e00780041
:10510000590207000000eb000080fa0000000600d2
:105110000600fa00000f78001e0078006101b90057
:105120001207980023079800300620000100200095
:105130001e019000ae019000800f5100818f590038
:10514000f6003e001e009000ae00900000600100de
:10515000630037006f0037007b003700870037009f
:10516000930037009f003700ab003700b7003700cf
:10517000c3003700cf003700e8003700e7003700f2
:10518000e6003700e5003700e4003700e3003700b1
:10519000e2003700e1003700e0003700df003700b1
:1051a000de003700dd003700dc003700db003700b1
:1051b000da003700d9003700d8003700d7003700b1
:1051c000d6003700d5003700d4003700d3003700b1
:1051d000d2003700d1003700d0003700cf003700b1
:1051e000ce003700cd003700cc003700cb003700b1
:1051f000ca003700c9003700c8003700c7003700b1
:10520000c6003700c5003700c4003700c3003700b0
:10521000c2003700c1003700c0003700bf003700b0
:10522000be003700bd003700bc003700bb003700b0
:10523000ba003700b9003700b8003700b7003700b0
:10524000b6003700b5003700b4003700b3003700b0
:10525000b2003700b1003700b0003700af003700b0
:10526000ae003700ad003700ac003700ab003700b0
:10527000aa003700a9003700a8003700a7003700b0
:10528000a6003700a5003700a4003700a3003700b0
:10529000a2003700a1003700a00037009f003700b0
:1052a0009e0037009d0037009c0037009b003700b0
:1052b0009a003700990037009800370097003700b0
:1052c00096003700950037009400370093003700b0
:1052d00092003700910037009000370082003700bd
:1052e0008000eb000000eb00df0107008000eb0016
:1052f00010002000dc0107008000eb0020002000ef
:10530000d90107008000eb0030002000d601070023
:105310008e003700110020000000eb00d2010700d2
:105320008000eb0010002000cf0107008000eb00a0
:1053300020002000cc0107008000eb00300020009e
:10534000c9010700810037008000eb000000eb007e
:10535000c50107001100200010002000c201070055
:105360008000eb0020002000bf0107008000eb0060
:1053700030002000bc01070074003700110020003d
:105380000000eb00b8010700110020001000200011
:10539000b50107008000eb0020002000b2010700eb
:1053a0008000eb0030002000af01070067003700ed
:1053b0008000eb000000eb00ab0107008000eb0079
:1053c00010002000a801070011002000200020008c
:1053d000a50107008000eb0030002000a2010700bb
:1053e0005a003700110020000000eb009e0107006a
:1053f0008000eb00100020009b010700110020003e
:1054000020002000980107008000eb003000200001
:10541000950107004d0037008000eb000000eb0015
:105420009101070011002000100020008e010700ec
:1054300011002000200020008b0107008000eb00fd
:1054400030002000880107004000370011002000d4
:105450000000eb0084010700110020001000200074
:105460008101070011002000200020007e010700bc
:105470008000eb00300020007b0107003300370084
:105480008000eb000000eb00770107008000eb00dc
:1054900010002000740107008000eb0020002000b5
:1054a0007101070011002000300020006e0107008c
:1054b00026003700110020000000eb006a01070001
:1054c0008000eb0010002000670107008000eb0067
:1054d000200020006401070011002000300020009f
:1054e0006101070019003700110020000000eb00e7
:1054f0005d01070011002000100020005a01070084
:10550000110020002000200057010700110020009a
:1055100030002000540107000c003700110020006b
:105520000000eb00500107001100200010002000d7
:105530004d01070011002000200020004a01070053
:105540001100200030002000470107000080fa0011
:10555000000006001000fa00500798000000eb0061
:10556000400798000000eb00300798000000eb00b7
:10557000200798006000b800008fbe005e00900019
:10558000e70f500002003400700020005007980020
:1055900060c2a9005e009000ddfe07000040eb0045
:1055a000610e0700400798000040eb005e0e070008
:1055b0003007980000000000a0002000d4fe070083
:1055c0004e009000200798002e0090004500dd005e
:1055d00020079800be009000800f2000008060002f
:1055e000300798003e0090004300de00300798002e
:1055f000be009000f00f2000808060002e00900020
:1056000001007000200798002e009000cf80de007f
:1056100058ec070060079800710798002e00900072
:105620000000e00007003d00020020000378240095
:105630006e009000fe0090007aec07006007980072
:10564000710798000200200003e823006e0090001c
:10565000fe009000d0ec0700008fbe001e01be00cf
:105660005e009000030007001e00be000080fa00ec
:10567000000006004e00fa00889fbe008a1f7800d6
:105680004027980052279800632798006800470039
:1056900001dd29000f000900311878000002b10077
:1056a0006000b800200798003107980080022000b1
:1056b0000e00400002db29000f00090032187800bc
:1056c0000002b1000000eb00100798000000eb00a2
:1056d000000f78004e2090008000400000802000e5
:1056e0000080400010007800f30f50002c003400c0
:1056f0000000eb00000f7800110037004e229000f0
:105700009e0278004e2090001e01e8007400b9004f
:1057100002004000c200dd00008120000080400047
:105720001001be007420b90005004000c200dd0079
:1057300000812000008040000288be001e0fe800ab
:10574000330120009e8f1100ecff34004e209000aa
:105750008000400000802000808040003001200058
:1057600080087800ce2190004e20900080004000fc
:105770000080200000804000100178007418b900fb
:1057800002004000c200dd000081200000804000d7
:105790005e219000ee2190000288be000e003700ce
:1057a000ce2190004e20900080004000008020001c
:1057b00000804000100178007418b9000200400019
:1057c000c200dd0000812000008040005e219000ca
:1057d000ee2190000288be000000eb001007980048
:1057e0001a0037004e2490004e20900081022000c5
:1057f0008e8040004200dd00010040001002be002b
:105800004e2090001e0190007400b900020040007c
:10581000c200dd0000812000008040001001be00b9
:105820000400be00ffeb07000001be008102200063
:105830008e8040004240dd00010040000288be0032
:105840001e0090000000e800100798004e20900015
:105850008000400000802000008040009000780020
:105860001e009000808f5000deff3d004e2590000e
:105870004e209000810220008e8040004200dd001a
:10588000010040001004be004e2090008000400047
:105890000080200000804000100078000000e80038
:1058a000cf80de00b3eb07000001be000800be00a1
:1058b0006dec07000001be00e80047004250dd002b
:1058c000010040000288be00ce209000018140000f
:1058d0000080200000004100100078000001e80076
:1058e0008180400000802000008040000208780095
:1058f0004e209000e80047004200dd00010040001b
:105900001001be0022079800330798004f05780069
:105910004f04be000080fa00000006000a00fa00f2
:105920002007980032079800430798006000b800ed
:10593000008fbe0002002c00934724003e00900020
:10594000ce0090008aec07000000e0000100320069
:10595000070037002e009000c200dd0000a92000e3
:1059600000804000301f78002017780007003700c3
:105970002e009000c200dd0000a920000080400041
:105980003e019000ce0190000288be001e00be00c5
:105990000080fa00000006000000fa000080eb0022
:1059a0006019880080072000c016880000082000c9
:1059b000001788000000eb00401788000000eb0093
:1059c000801788006da0a90000000000ec82a900eb
:1059d00000000000eca2a90000000000ecc2a90039
:1059e00000000000f442a90000000000e4c2a90089
:1059f00000000000ec02a90000000000ec22a90059
:105a000000000000ec42a90000000000ec62a900c8
:105a100000000000e4a2a90000000000e482a80049
:105a200000000000e462a90000000000e442a900b8
:105a300000000000e422a90000000000e402a90028
:105a400000000000dc02a90000000000dc22a90028
:105a500000000000dc42a90000000000dd62a80098
:105a60000080fa00000006000800fa00000f78002d
:105a7000110798001e0090000000e00002003200b4
:105a80001000200010079800000000001e007800a1
:105a90006101b90022079800330798002001200017
:105aa000010020002e019000be019000800f5100e7
:105ab000818f5900e3003e002e009000be00900050
:105ac00000600100120037001c003700260037007c
:105ad000300037003a003700440037004d003700ef
:105ae00057003700610037006b0037007500370042
:105af0007f00370089003700930037009d00370092
:105b0000a6003700af003700b9003700c3003700e8
:105b10001e00900061406000614060004401dd00b3
:105b2000c12e200091407800f0ceb30000c060008c
:105b300002407000ece2b700c20037001e00900087
:105b400061406000614060004501dd00c12e200021
:105b500091407800f0cdb30000c0600002407000ba
:105b6000ece2b700b70037001e0090006140600013
:105b7000614060004601dd00c12e200091407800a8
:105b8000f0cbb30000c0600002407000ece2b70050
:105b9000ac0037001e009000614060006140600072
:105ba0004201dd00412f200091407800b0cfb300ca
:105bb00000c0600002407000f4e2b700a1003700ae
:105bc0001e00900061406000614060004601dd0001
:105bd000412e200091407800f0cbb30000c060005f
:105be00002407000e4e2b700960037001e0090000b
:105bf0006140600061416000c12e2000914078004a
:105c0000e0cfb30000c0600002407000ece2b700db
:105c10008c0037001e009000614060006140600011
:105c200000414000c12e200091407800d0cfb30049
:105c300000c0600002407000ece2b7008100370055
:105c40001e00900061406000614060004201dd0084
:105c5000c12e200091407800b0cfb30000c060009a
:105c600002407000ece2b700760037001e009000a2
:105c700061406000614060004301dd00c12e2000f2
:105c80009140780070cfb30000c060000240700007
:105c9000ece2b7006b0037001e009000614060002e
:105ca000614060004501dd00412e200091407800f8
:105cb000f0cdb30000c0600002407000e4e2b70025
:105cc000600037001e00900061406000614060008d
:105cd0004401dd00412e200091407800f0ceb30059
:105ce00000c0600002407000e4e2b70055003700d9
:105cf0001e00900061406000614060004301dd00d3
:105d0000412e20009140780070cfb30000c06000a9
:105d100002407000e4e2b7004a0037001e00900025
:105d200061406000614060004201dd00412e2000c2
:105d300091407800b0cfb30000c060000240700016
:105d4000e4e2b7003f0037001e00900061406000b1
:105d50006140600000414000412e200091407800e9
:105d6000d0cfb30000c0600002407000e4e2b70092
:105d7000340037001e009000614060006141600007
:105d8000412e200091407800e0cfb30000c06000b9
:105d900002407000e4e2b7002a0037001e009000c5
:105da0006140600061416000c12d20009140780099
:105db000e0cfb30000c0600002407000dce2b7003a
:105dc000200037001e0090006140600061406000cc
:105dd00000414000c12d200091407800d0cfb30099
:105de00000c0600002407000dce2b7001500370020
:105df0001e00900061406000614060004201dd00d3
:105e0000c12d200091407800b0cfb30000c06000e9
:105e100002407000dce2b7000a0037001e0090006c
:105e200061406000614060004301dd00d12d200031
:105e30009140780070cfb30000c060000240700055
:105e4000dde2b7000080fa00000006000800fa005a
:105e5000000f7800000000000000eb00a08f880019
:105e60001e0078006101b9002207980033079800ee
:105e700020012000010020002e019000be019000b2
:105e8000800f5100818f590095003e002e00900038
:105e9000be009000006001001200370018003700bb
:105ea0001e003700240037002a003700300037007a
:105eb000340037003a003700400037004600370012
:105ec0004c00370052003700580037005e003700a2
:105ed00064003700680037006c003700720037003c
:105ee00078003700ecc2bf000080fb004400de00f9
:105ef000614060000080fb00100798007a003700c6
:105f0000ecc2bf000080fb004500de006140600085
:105f10000080fb001007980073003700ecc2bf0040
:105f20000080fb004600de00614060000080fb0056
:105f3000100798006c003700f4c2bf000080fb001f
:105f40004200de00614060000080fb001007980006
:105f500065003700e4c2bf000080fb004600de00a1
:105f6000614060000080fb00100798005e00370071
:105f7000ecc2bf00614060000080fb001007980089
:105f800059003700ecc2bf000080fb000000d100c8
:105f9000614060000080fb0010079800520037004d
:105fa000ecc2bf000080fb004200de0061406000e8
:105fb0000080fb00100798004b003700ecc2bf00c8
:105fc0000080fb004300de00614060000080fb00b9
:105fd0001007980044003700e4c2bf000080fb00b7
:105fe0004500de00614060000080fb001007980063
:105ff0003d003700e4c2bf000080fb004400de002b
:10600000614060000080fb001007980036003700f8
:10601000e4c2bf000080fb004300de00614060007e
:106020000080fb00100798002f003700e4c2bf007b
:106030000080fb004200de00614060000080fb0049
:106040001007980028003700e4c2bf000080fb0062
:106050000000d100614060000080fb001007980044
:1060600021003700e4c2bf00614060000080fb00f7
:10607000100798001c003700dcc2bf0061406000c0
:106080000080fb001007980017003700dcc2bf003b
:106090000080fb000000d100614060000080fb0038
:1060a0001007980010003700dcc2bf000080fb0022
:1060b0004200de00614060000080fb001007980095
:1060c00009003700ddc2bf000080fb004300de0096
:1060d000614060000080fb0010079800020037005c
:1060e0008000eb00110798001e0090000080fa006d
:1060f000000006000600fa002007980010002000ab
:10610000000f78000000eb00100798000b0037002c
:106110002e0090001e006000800078001e0090009d
:1061200051fe07001e00780000004000000f7800bc
:106130001e0090000000e800100798001e0090006c
:10614000f20f5000f2ff34000080fa000000060059
:106150000600fa0010002000100798000000eb0075
:10616000000f78000000eb00200798000c003700bb
:106170002e00900035ff07000000e0000200320012
:106180001e0090001e0f40001e0090000000400006
:10619000100798002e0090000000e80020079800eb
:1061a0002e009000f20f5000f1ff34001e00780026
:1061b0000080fa00000006000800fa00000f7800d6
:1061c000000000000000eb00a08f88001e00780097
:1061d0006101b9002207980033079800f000200001
:1061e000010020002e019000be019000800f5100a0
:1061f000818f590056003e002e009000be00900096
:10620000006001000f003700150037001b00370049
:1062100021003700270037002c0037002e00370000
:1062200030003700320037003400370036003700c6
:10623000380037003a0037003c0037003e00370096
:1062400040003700dac2bf000080fb004300de00e0
:10625000614060000080fb00100798003e0037009e
:10626000dac2bf000080fb004400de006140600035
:106270000080fb001007980037003700dac2bf002b
:106280000080fb004500de00614060000080fb00f4
:106290001007980030003700dac2bf000080fb0012
:1062a0004600de00614060000080fb00100798009f
:1062b00029003700e2c2bf000080fb004700de007b
:1062c0000080fb001007980023003700a18f80009a
:1062d0001107980020003700a28f80001207980055
:1062e0001d003700a38f8000130798001a003700a5
:1062f000a08f80001007980017003700a18f800042
:106300001107980014003700a28f80001207980030
:1063100011003700a38f8000130798000e0037008c
:10632000a08f8000100798000b003700a18f80001d
:106330001107980008003700a28f8000120798000c
:1063400005003700a38f8000130798000200370074
:106350000000eb00100798001e0090000080fa007b
:10636000000006000600fa00100020001007980048
:106370000000eb00000f78000000eb002007980001
:106380000c0037002e0090008bff07000000e0009b
:10639000020032001e0090001e0f40001e00900000
:1063a00000004000100798002e0090000000e80058
:1063b000200798002e009000ef0f5000f1ff3400ee
:0c63c0001e0078000080fa0000000600bb
:020000040000fa
:1063cc00761000008e0000000000000000080000a5
:1063dc00f00200000000000004110000500000005a
:1063ec00020000000000000000000000000000009f
:1063fc000000000000000000000000000000000091
:10640c000000000000000000000000000000000080
:10641c000000000000000000000000000000000070
:10642c000000000000000000000000000000000060
:10643c000000000000000000000000000000000050
:10644c000000000000000000000000000000000040
:10645c00f01100000200000000000000f21100002a
:10646c000200000000000000ea110000060000001d
:10647c0000000000f4110000020000000000000009
:10648c00100d00005e01000000000000541100001f
:10649c004000000000000000d411000016000000b5
:1064ac0002000000000000000000000000000000de
:1064bc0000000000000000000000000000000100cf
:1064cc00000000006e0e000008010000000000003b
:1064dc00760f0000000100000200000029b3090043
:1064ec00285de000185e27006e465500c481500000
:1064fc000b7f2a005708f30060ae99003dc01100d5
:10650c0014eb07002fde3500d86570002c8b6d0066
:10651c00e96c3900f0e5a000dbfb0f00ddf5ef00c6
:10652c0068b621008a3ba600f792be001f7dbc0016
:10653c00726156009d6a03008e42450098b174004a
:10654c003295f200901c1d005f25020075f641008b
:10655c00b7cef100e6830d00913f6200c8b0e200b7
:10656c00059ebd00311236001e78e30044305b00fe
:10657c0059fcd200b9cb8c00ab9b3800a2f9c900f6
:10658c0086f44300c594f800526422005aec3300a0
:10659c00a7b2cf00c1a4e100da934f0047d997000e
:1065ac0026c6d700d47b9c004c797100fd37ff00c8
:1065bc001719e700bb154800d1675100230c0600e2
:1065cc007a4e20003c5c0e00ca538000c387df006b
:1065dc00d3b554000077ad00a5ea2d00d06b880030
:1065ec00c77e8d00a3b46300acdc4b0073e86f0076
:1065fc00e4cced0049fe3e006984160024768f0041
:10660c00a185a9000a34ba00b8aa4d00cd897c0036
:10661c00ee109f00fabf4a001b820400c2012e003c
:10662c003a664000a8965800d6afd5009a1a2b00af
:10663c0000000000f00a0000200200000200000030
:10664c00000000000000000000000000000000003e
:10665c00000000000000000000000000000000002e
:10666c00000000000000000000000000000000001e
:10667c00000000000000000000000000000000000e
:10691c000000000000000000941100004000000086
:10692c000000000056130000a00000000200000050
:10693c00010000000000000000000a000000000040
:10694c0000000000006400000000000000000000d7
:10695c00e803000000000000000010002700000009
:10696c000000000000a086000100000000000000f4
:10697c0040420f00000000000000800096980000cc
:10698c00000000000000e100f50500000000000020
:10699c0000ca9a003b00000000000000e40b540009
:1069ac00020000000000e80076481700000000001c
:1069bc000010a500d4e8000000000000a0724e00fa
:1069cc0018090000000040007a10f3005a00000083
:1069dc000080c600a47e8d000300000000c16f0083
:1069ec00f2862300000000008a5d780045630100f8
:1069fc0000006400a7b3b600e00d000000e88900b9
:106a0c000423c7008a000000f61300002a000000cf
:106a1c0002000000286e75006c6c290000303100fb
:106a2c0032333400353637003839410042434400a4
:106a3c0045460000303132003334350036373800eb
:106a4c00396162006364650066000000f6110000a5
:106a5c0060010000020000000000000000000000c7
:106a6c00f03f00000000a0009999b9003f00000021
:106a7c000040e1007a843f0000000000e04d62001d
:106a8c00503f00000000e000e2361a003f0000001a
:106a9c000080b500f8e43e0000000000a0f7c6003e
:106aac00b03e00000000a000f2d77a003e000000cb
:106abc0000e08e0079453e0000000000e00b2e0047
:106acc00113e00000000e000df7cdb003d00000018
:106adc000000a1009cc73b0000000000004c4800d7
:106aec00b439000000000000206ca1003700000049
:106afc00000000000000000000000000000000008a
:106b0c000000000000000000000000000000000079
:106b1c000000000000000000000000000000000069
:106b2c000000000000000000000000000000000059
:106b3c000000000000000000000000000000000049
:106b4c0000000000000000000000f0003f0000000a
:106b5c0000000000002440000000000000000000c5
:106b6c00594000000000000000408f004000000071
:106b7c000000000088c340000000000000006a0014
:106b8c00f84000000000000080842e00410000004e
:106b9c000000d00012634100000000000084d70008
:106bac00974100000000000065cdcd0041000000c1
:106bbc0000205f00a002420000000000801daf001a
:106bcc001544000000004000593e2900460000001a
:106bdc000000000000f07f0000000000000000003a
:106bec00f07f0000000000000000f0007f000000bb
:106bfc000000000000f07f0000000000000000001a
:106c0c00f07f0000000000000000f0007f0000009a
:106c1c000000000000f07f000000000000000000f9
:106c2c00f07f0000000000000000f0007f0000007a
:106c3c00201400002600000002000000221448006e
:106c4c001400000048140900000000000200460077
:106c5c0014000000461406000201000000000000b1
:106c6c00000000000000060002020000000000000e
:106c7c004614000006000000000000004c14000048
:106c8c0002000000020000000100000000000000f3
:020000040000fa
:106c9c000000fa0041d22000c0d220008008780009
:106cac0041d220000000eb009000980041d220005f
:106cbc000000eb00a000980041d22000f001200061
:106ccc00b0009800012420009140780030ceb30031
:106cdc0000c060000024a00040e2b7004342a800be
:106cec0042e2a80042a2a900212420009140780091
:106cfc0030ceb30000c060008041b30042e2b70068
:106d0c0042c2bf003040b30042e2b7004402a900c7
:106d1c0040c2a90041e2a8008540a900a9c0bf005b
:106d2c007040b300a9e0b7009540a8000080fa00bd
:106d3c00000006000400fa0010079800d8080700ad
:106d4c0041d220001e00900008030700000f7800bd
:106d5c00dd0807001e0078000080fa000000060025
:106d6c000000fa00d06880000080fa0000000600e5
:106d7c000000fa00e06880000080fa0000000600c5
:106d8c000000fa00006980000080fa000000060094
:106d9c000000fa00f06880000080fa000000060095
:106dac000000fa00106980000080fa000000060064
:106dbc000000fa00906880000080fa0000000600d5
:106dcc000000fa000000eb00d06888000080fa0098
:106ddc00000006000000fa000000eb00e0688800ec
:106dec000080fa00000006000000fa000000eb0032
:106dfc00006988000080fa00000006000000fa001c
:106e0c000000eb00f06888000080fa00000006002b
:106e1c000000fa000000eb00106988000080fa0006
:106e2c00000006000000fa000000eb0090688800eb
:106e3c000080fa00000006000601fa00806880005d
:106e4c000000e0002c0032006600470001df290042
:106e5c00ff000900315878000010b1000000eb0071
:106e6c0010079800090037001e0190002e009000ba
:106e7c00804078006600470000004100014878001f
:106e8c001e0090000000e800100798006400470006
:106e9c0041d22000b50207000000e000f2ff3a00ea
:106eac0040d22000d4020700c0d6200002102000df
:106ebc008000eb009eeb07006600470001ef290005
:106ecc004f040700000f78001e0078001040780077
:106edc000004e000040032004200200041f22900ce
:106eec001e0078009b0407000000eb0090688800ef
:106efc000000eb00806888000080fa0000000600ab
:106f0c00809fbe000800fa00cc82a80040128000ce
:106f1c0020079800ae00900061738800d068800054
:106f2c000000e800d0688800b06880000000e00035
:106f3c0087003a002e0090004a00de0010079800ef
:106f4c00ae009000f03f2000008f60001e00780023
:106f5c00c06888009e009000310798003e009000a9
:106f6c00e40f50003b003200be009000e48f500054
:106f7c000a003e003e009000e20f50002300320059
:106f8c00be009000e28f50002f003e003e009000ab
:106f9c00e10f50000b0032004d003700be00900096
:106fac00e68f5000330032003e009000e60f500098
:106fbc002c003900be009000e78f50003e003200dc
:106fcc004300370010002000b068880070102000cb
:106fdc009e0f10000a003e00c06880008000780000
:106fec00e0e6200000804000104078008080fb002c
:106ffc000040200000804000401288007b003700d9
:10700c000000eb00401288007800370020002000c0
:10701c00b0688800f00f20009e0f100007003e00a3
:10702c00c06880008000400000af2000008040005d
:10703c0010007800401288006c0037000000eb0054
:10704c00401288006900370030002000b0688800ca
:10705c0066003700e06880000000e800e068880007
:10706c0062003700e06880000000e800e0688800fb
:10707c005e003700806880000000e0000b003a00e2
:10708c00c1688000f00f2000808f500007003e0088
:10709c00c1688000c0d620000080400010407800fd
:1070ac000000fb0040128800500037000000eb008d
:1070bc00401288004d003700f03f20009e0f10005a
:1070cc0003003a0010002000806888004700370059
:1070dc00e06880000000e800e068880040d22000f2
:1070ec00100090008000e80040d22000300090009a
:1070fc008080600040d2200020009000808f5000e3
:10710c0003003a0010002000906888003700370018
:10711c0040d220009000780040d220001000900057
:10712c0000004000008040001e08780040d2200083
:10713c00100090008000e80040d220003000900049
:10714c008080600040d2200011009800270037009a
:10715c00b0688000e10f500006003a000069800022
:10716c000000e800006988000000eb00b0688800af
:10717c001e003700b0688000e20f500006003a0095
:10718c00f06880000000e800f06888000000eb0068
:10719c00b068880015003700b0688000e30f50001d
:1071ac0010003a00c1688000f00f2000808f500062
:1071bc0006003e00c06880008000400000af200048
:1071cc0000804000ae00900001087800106980003b
:1071dc000000e800106988000000eb00b06888002f
:1071ec00020037000000eb00b0688800cc82a900d8
:1071fc008540a9000080fa004f00be000040060048
:10720c000200fa000000eb00000f780027003700a6
:10721c009e0178001e0078004700dd008000780099
:10722c00200821000080400000017800a107210007
:10723c004318dd0001004000020878001e007800b1
:10724c00a10721004300dd000080e8008100400020
:10725c000000eb00800878001e007800a1072100d8
:10726c004300dd0064004000810040000000eb00a2
:10727c00800878001e007800a10721004300dd0083
:10728c006600400081004000f00720008008780074
:10729c001e007800800040002010210080804000fb
:1072ac000000eb00800878001e0fe8001e00e000d4
:1072bc00d7ff3400b00020004011880021e2a80064
:1072cc0020a2a9002062a900004020001011880013
:1072dc008560a9008580a900910a20009140780062
:1072ec00f0c8b30000c0600001c6b30001407000dc
:1072fc00a9e0b700a10a20009140780080cfb3002c
:10730c0000c060000014a000aae0b7009560a800bf
:10731c009580a9000080fa00000006000800fa0021
:10732c0010079800210798001e009000e10f5000f4
:10733c00010032000e003700590707001e009000b4
:10734c004300dd0080007800a00721006800500099
:10735c00808040002e0090000a010700000f78008a
:10736c00590707001e007800300798000500370009
:10737c00ae0090000040eb00804878000000eb006d
:10738c00300798003e0090000080fa0000000600d4
:10739c000800fa0010079800414798001e00900062
:1073ac00e10f5000010032000700370023c2bf007c
:1073bc000080fb000000d100614060000080fb00f9
:1073cc00000f78000200370010002000000f78003a
:1073dc001e00e0000a003a001e009000e10f500071
:1073ec0001003200060037004e4090000080fb0088
:1073fc002011880010002000300798000200370090
:10740c000000eb00300798003e0090000080fa006e
:10741c00000006000600fa001007980021079800eb
:10742c000000eb00000f78000b0037001e00780006
:10743c00800078002e009000008040001040780002
:10744c00804078001e009000d1ff07000000e00093
:10745c00010032001e0fe8001e007800800078004a
:10746c002e00900000804000104078000004e000e6
:10747c00eeff3a000000eb000080fa00000006006e
:10748c000600fa00100798001e009000e10f500053
:10749c00010032000d003700010707001e009000ac
:1074ac004300dd0080007800a00721006800500038
:1074bc0000804000df000700000f78000207070083
:1074cc001e00780020079800020037000000eb0037
:1074dc00200798002e0090000080fa0000000600a3
:1074ec000400fa00100798001e009000e10f5000f5
:1074fc00010032000700370023c2bf000080fb00f0
:10750c000000d100614060000080fb00000f78009b
:10751c000200370010002000000f78001e007800d9
:10752c000080fa00000006000400fa00000f78004a
:10753c001e007800e10f50000100320007003700f8
:10754c001e007800800040002010210000804000c8
:10755c001000780010079800020037000000eb00c4
:10756c00100798001e0090000080fa000000060032
:10757c000200fa00000f78001e007800e10f5000a6
:10758c0001003200060037001e0078008000400029
:10759c0020102100808040000000eb008008780063
:1075ac000080fa00000006000400fa0010079800a2
:1075bc001e009000e10f5000010032001300370054
:1075cc00b70607001e0090004300dd008000780025
:1075dc00a007210068005000008040008b000700cd
:1075ec001e009000e10f500003003200060037002f
:1075fc0030118000000f780022c2bf006140600093
:10760c000004e000faff3a00af0607000080fa0021
:10761c00000006000200fa00000f78001e0078003f
:10762c00e10f500001003200040037002342a90092
:10763c00000000002342a800000000000080fa00b7
:10764c0000000600809fbe000000fa00b08380009e
:10765c00c183800061004000e0804800b083880056
:10766c00c18388008580a9000080fa004f00be000d
:10767c0000400600809fbe000000fa001c0037008e
:10768c00a0072100100090008000e800a007210056
:10769c003000900080806000a00721002000900046
:1076ac00808f500003003a001000200010888800e2
:1076bc000f003700a007210090007800a0072100e0
:1076cc0010009000808040003011800080487800cd
:1076dc00a0072100100090008000e800a007210006
:1076ec003000900080806000a007210011009800fd
:1076fc0022c2bf00614060000004e000e0ff3a00dd
:10770c008560a9000080fa004f00be000040060012
:10771c000600fa00004f7800110798001e00900038
:10772c00440007000000e000030032000000eb0002
:10773c0020079800100037001e0090009000780081
:10774c001e00900010009000008040001e48780041
:10775c001e009000100090008000e8001e009000b9
:10776c0030009000808060001e0090001100980096
:10777c0010002000200798002e0090000080fa00d6
:10778c00000006000600fa00000f780011079800b0
:10779c001e0090003b0007000000e00006003200d5
:1077ac009e0078000040eb00804878000000eb0061
:1077bc0020079800120037001e00900090007800ff
:1077cc001e00900020009000008040009040780047
:1077dc001e007800014878001e00900020009000e8
:1077ec008000e8001e009000300090008080600057
:1077fc001e00900021009800100020002007980027
:10780c002e0090000080fa00000006000200fa0032
:10781c00000f78009e0078000000eb00a00098009c
:10782c009e0078000000eb00900098000080fa00a9
:10783c00000006000400fa00000f78001e0078001b
:10784c00100090008000e8001e00780030009000ce
:10785c00808060001e00780020009000808f500017
:10786c0003003a00100020001007980002003700b7
:10787c000000eb00100798001e0090000080fa003a
:10788c00000006000400fa00000f78001e007800cb
:10789c00a00090001e00780010009000808f500017
:1078ac0003003a0010002000100798000200370077
:1078bc000000eb00100798001e0090000080fa00fa
:1078cc00000006000200fa00000f78001e0078008d
:1078dc00900090001e0078002000900080805000e6
:1078ec001e00780030009000008060000080fa00dc
:1078fc00000006000600fa00000f7800110798003f
:10790c001e009000460007000000e000030032005b
:10791c000000eb0020079800110037001e009000bb
:10792c00900078001e0090001000900000004000b5
:10793c00008040001e0878001e009000100090008f
:10794c008000e8001e0090003000900080806000f5
:10795c001e009000110098001000200020079800d5
:10796c002e0090000080fa00000006000600fa00cd
:10797c00000f7800110798001e0090003c000700d3
:10798c000000e000060032009e0078000000eb00d2
:10799c00800878000000eb002007980013003700e7
:1079ac001e009000900078001e00900020009000b7
:1079bc000000400000804000900078001e0078001d
:1079cc00010878001e009000200090008000e80064
:1079dc001e00900030009000808060001e0090001f
:1079ec002100980010002000200798002e00900025
:1079fc000080fa00000006000200fa00000f780078
:107a0c009e0078000000eb00a00098009e0078001b
:107a1c000000eb00900098000080fa0000000600c7
:107a2c000400fa00000f78001e007800100090008f
:107a3c008000e8001e00780030009000808060001c
:107a4c001e00780020009000808f500003003a0048
:107a5c001000200010079800020037000000eb0017
:107a6c00100798001e0090000080fa00000006002d
:107a7c000400fa00000f78001e007800a0009000af
:107a8c001e00780010009000808f500003003a0018
:107a9c001000200010079800020037000000eb00d7
:107aac00100798001e0090000080fa0000000600ed
:107abc000200fa00000f78001e0078009000900081
:107acc001e00780020009000808050001e0078007e
:107adc0030009000008060000080fa00000006007a
:107aec004800fa00201f9800311f9800421f980090
:107afc006400470081102a00170009003118780033
:107b0c000003b1004e19900032279800be2190005e
:107b1c00e18f5100430032003e209000e20f5000f4
:107b2c007c003200be2090000100e0000100320019
:107b3c00b4003700640147000000200001f8230066
:107b4c000089be00640147000000200001f82300fa
:107b5c0020019800310198006401470000002000ca
:107b6c0001f823004001980051019800640147007e
:107b7c000000200001f823006001980071019800ba
:107b8c00640147000000200001f823000009980060
:107b9c0011099800640147000000200001f823003f
:107bac00200998003109980064014700000020006a
:107bbc0001f823004009980051099800640147001e
:107bcc000000200001f8230060099800710998005a
:107bdc00640147000000200001f823000011980008
:107bec0011119800640147000000200001f82300e7
:107bfc00201198003111980064014700000020000a
:107c0c0001f82300401198005111980064014700bd
:107c1c000000200001f823006011980071119800f9
:107c2c007d003700640147008000200001822300a2
:107c3c000089be00640147008000200001822300ff
:107c4c002001980031019800640147008000200059
:107c5c000182230040019800510198006401470003
:107c6c0080002000018223006001980071019800bf
:107c7c006401470080002000018223000009980065
:107c8c001109980064014700800020000182230044
:107c9c0020099800310998006401470080002000f9
:107cac0001822300400998005109980064014700a3
:107cbc00800020000182230060099800710998005f
:107ccc00640147008000200001822300001198000d
:107cdc0011119800640147008000200001822300ec
:107cec002011980031119800640147008000200099
:107cfc000182230040119800511198006401470043
:107d0c0080002000018223006011980071119800fe
:107d1c004100370064014700a000200081ac230023
:107d2c000089be0064014700a000200081ac230044
:107d3c00200198003101980064014700a000200048
:107d4c0081ac230040019800510198006401470068
:107d5c00a000200081ac2300600198007101980004
:107d6c0064014700a000200081ac230000099800aa
:107d7c001109980064014700a000200081a4230091
:107d8c00200998003109980064014700a0002000e8
:107d9c0081ac230040099800510998006401470008
:107dac00800020000182230060099800710998006e
:107dbc006401470070002000017823000011980036
:107dcc001111980064014700700020000178230015
:107ddc0020119800311198006401470070002000b8
:107dec00017823004011980051119800640147005c
:107dfc00800020000182230060119800711198000e
:107e0c00050037000200200003f82b001227980011
:107e1c00232798001f0037002e189000e40047001d
:107e2c004200dd00010040001001be00721f9800ee
:107e3c00032798003e189000cf80de004ae207002e
:107e4c00501f9800611f98003e1890000000e00041
:107e5c0007003d0002002000037824005e1890000b
:107e6c00ee1890006ce20700501f9800611f9800fc
:107e7c005e199000ee1990007e1890008e209000f4
:107e8c00c2e20700008fbe001e00be001027980043
:107e9c00212798001e209000ae2090000080fa0050
:107eac00000006000800fa00881f780010079800f0
:107ebc00210798000000eb00000f78001e009000d6
:107ecc00104078000004e00003003a000000eb00d2
:107edc0030079800460037001e00780080007800bc
:107eec002e00900000804000104078000000fb0045
:107efc00b0e10700000478001e00780080007800d4
:107f0c001e00900000804000104078000000fb0034
:107f1c00a8e10700800f5400150032002e009000dd
:107f2c000000e800200798002e0090001040780018
:107f3c000004e00003003a000000eb00300798005a
:107f4c002b0037002e00900090407800c0c7b30083
:107f5c0080cf5000f1ff3a002e0090000000e800a6
:107f6c00200798000000eb00000f78001b00370082
:107f7c001e0fe8001e007800800078002e00900094
:107f8c0000804000104078000004e000080032003f
:107f9c001e007800800078002e00900000804000c9
:107fac0090407800c0c7b30080cf50000b003a005f
:107fbc001e007800800078001e00900000804000b9
:107fcc0010407800520007000000e00003003a0067
:107fdc001e00780030079800050037007002200062
:107fec009e0f1000bcff34001e0078003007980074
:107ffc003e0090004f0478000080fa00000006005c
:10800c000600fa0010079800210798000080eb008a
:10801c00000f78000e0037001e0090001041780011
:10802c001e007800800078002e0090000080400038
:10803c0010407800804f510005003a001e0090005f
:10804c000000e800100798000080eb00000f78009b
:10805c001e0fe8001e007800800078002e009000b3
:10806c0000804000104078000004e000eaff3a0075
:10807c001e0090000080fa00000006000400fa00c8
:10808c00000f780081132a001e007800dcff070027
:10809c00000f78001e00780090407800d0c2b3002a
:1080ac0080cf5000050032001e0078009040780010
:1080bc00b0c2b30080cf500001003a001e0fe800a0
:1080cc00b1132a001e007800cdff0700000f7800c6
:1080dc00d1132a001e007800c9ff0700000f78009a
:1080ec001e007800104078000004e000030032000d
:1080fc000000eb0010079800020037001000200071
:10810c00100798001e0090000080fa000000060086
:10811c000400fa00004f78001e00fb002ce1070061
:10812c000000e00003003a00f0c5b3009e4f1000c1
:10813c0003003a00100020001007980002003700de
:10814c000000eb00100798001e0090000080fa0061
:10815c00000006000c00fa00200798003107980078
:10816c00420798000000eb00000f780081132a00f2
:10817c002e009000a2ff0700200798001e00370079
:10818c001e0078004200dd00800078003e00900068
:10819c0000804000900078002e00900041ff070006
:1081ac00100798001e0090000000e0001100320043
:1081bc001e009000800078002e009000008040008f
:1081cc0081132a008eff0700200798001e007800fc
:1081dc004200dd00800078003e00900000804000ee
:1081ec00900090002e0090000100010050079800b4
:1081fc000c0037001e0fe8001e0078004200dd0066
:10820c00800078003e009000008040001000780054
:10821c00104078000004e000d9ff3a004e009000b6
:10822c00500798005e0090000080fa0000000600e5
:10823c000000fa000000eb00800888000000eb0052
:10824c0030088800f07f24006008880084e0a900d2
:10825c0094e0a80011e1a8000080fa0000000600dc
:10826c000000fa00b30007000080fa0000000600ce
:10827c000200fa00000f78001e0078001000780051
:10828c000080fa00000006000200fa00000f7800df
:10829c001e007800640007001e0078000200070032
:1082ac000080fa00000006000200fa00000f7800bf
:1082bc001e0178006000b800300198004101980060
:1082cc00960007001e01780010019800210198000b
:1082dc000080fa00000006000600fa002007980053
:1082ec008e000700008fbe002e009000100078005a
:1082fc000000e000230032002e009000a00090004f
:10830c0010009000be0f5000ae8f58000f003600ca
:10831c002e00900030019000c00190002e009000c3
:10832c00a0009000100090003e024000ae82480079
:10833c000400be0002004000838048002e01900023
:10834c0030019800410198000e0037002e0090007b
:10835c0030019000c00190002e009000a000900011
:10836c00100090003e021000ae8218000400be0007
:10837c0002004000838048002e01900030019800dc
:10838c00410198002e0090001e01be0012009800c2
:10839c00230098002e00900030039000c003900042
:1083ac0086007800a0002000000ab8006030b900f8
:1083bc0005017800000141006a38b9000001410054
:1083cc00820278000400be000080fa000000060063
:1083dc000200fa00000f78001e007800beff0700b4
:1083ec009e00780010002000800878001e007800a5
:1083fc0030039000c003900086007800a00020009d
:10840c00000ab8006030b900050178000001410095
:10841c006a38b90000014100820278000400be00f5
:10842c000080fa00000006000200fa00000f78003d
:10843c001e007800a8ff07009e0078000000eb00eb
:10844c00800878001e00780030039000c003900074
:10845c0086007800a0002000000ab8006030b90047
:10846c0005017800000141006a38b90000014100a3
:10847c00820278000400be000080fa0000000600b2
:10848c000600fa0020079800240007000001be0037
:10849c002e00900001002000001f410001974900b0
:1084ac001e000700be0f5000ae8f5800fcff3900b5
:1084bc000080fa00000006000600fa002007980071
:1084cc0016000700008fbe002e009000e90f500030
:1084dc00080036002e009000a200200011000900b8
:1084ec000280d800010020001e0f40005e9748005b
:1084fc000400370010002000010020001e0f400077
:10850c005e97480005000700be0f5000ae8f580064
:10851c00fcff39000080fa00000006000000fa00a1
:10852c0004000700608f8000718f80000080fa00cb
:10853c00000006000200fa00528f8000608f80005d
:10854c00718f8000000f51001e0078006101b8008f
:10855c00608f8000718f8000020040008380480093
:10856c00608f8800718f88000080fa000000060080
:10857c00801f78000000fa000000eb003008880033
:10858c00508f80000000e800508f880084e0a90024
:10859c000080fa004f007800004006000a00fa0044
:1085ac001007980041479800320798001e00900071
:1085bc000000e000030032003e0090000000e000ec
:1085cc0003003a00100020004007980034003700e8
:1085dc001e009000dde50700000f78009e80e8008b
:1085ec00f00f2000808f5000030036001000200098
:1085fc00400798002a0037003e009000e70040003a
:10860c003e009000704092000080fb000080400013
:10861c009e009000d3e507003e009000f0409200d1
:10862c001e00780080c040003e00900071409a000f
:10863c003e009000e70040003e0090007040920029
:10864c000080fb00808040000040eb0080487800f8
:10865c003e009000704092008040e8003e00900088
:10866c0071409a003e009000e70040003e009000f0
:10867c00704092000080fb00808040004e409000d3
:10868c00804878003e009000704092008040e800e6
:10869c003e00900071409a000000eb0040079800eb
:1086ac004e0090000080fa00000006001c00fa004a
:1086bc00400f98000000eb00200798004e08900037
:1086cc000000e000610032004e089000104078007d
:1086dc000080fb00801f7800400b2a00801f780070
:1086ec0040152100bee50700e48757004115210025
:1086fc001000200047fb07004e0890000000e80027
:10870c00801f7800400c2a00801f78004015210043
:10871c00b3e50700e4875700411521001000200045
:10872c003cfb0700410d2a001000200039fb07001c
:10873c000000eb00300798003e0037004e08900018
:10874c00e70040002e009000808040006800470049
:10875c00020120008be5070091c0b300100020003f
:10876c000bfb0700e80047001000200029fb070066
:10877c006800470075e50700800078002e00900027
:10878c0001004000200798002e0090000000e80037
:10879c00200798002e009000ce0890006600400044
:1087ac0001004000104090000000fb0010079800f2
:1087bc002e0090000000e800200798001e0090009a
:1087cc00500f98005e089000e20f50000b00320032
:1087dc005e089000e30f50000c0032005e08900021
:1087ec00e10f5000010032000c003700610e2a002e
:1087fc001000200007fb07000b003700010f2a00b8
:10880c001000200003fb070007003700b10f2a00ff
:10881c0010002000fffa07000300370051102a0057
:10882c0010002000fbfa07003e0090000000e8005a
:10883c00300798004e089000604090008080fb004c
:10884c003e009000808f5000bcff3e000080fa007c
:10885c00000006008e00fa000000eb0010079800e4
:10886c00416a20009140780000ccb30000c0600049
:10887c003040b300a4e6b700416c20009140780072
:10888c0000ccb30000c060003040b300c4e6b700b9
:10889c00816a20009140780000ccb30000c06000d9
:1088ac005041b300a8e6b700a16d200091407800bc
:1088bc0000ccb30000c060007040b300dae6b70033
:1088cc00316d20009140780000ccb30000c06000f6
:1088dc000034a000d3e6b700a16a200091407800d4
:1088ec0000ccb30000c06000b041b300aae6b700f2
:1088fc0026f4070042fa07004dfe0700e4f80700d3
:10890c004301070075000700ea004700c0052a0074
:10891c00801f780050062a00801f780010072a005c
:10892c00801f7800010078002de50700e6875700ce
:10893c00ea00470010002000b6fa0700a00720004c
:10894c000e00400058fe0700a00720000e0040005b
:10895c009ffe0700400820000e00400052fe07005a
:10896c00400820000e00400099fe0700f462a800a9
:10897c000000eb00000f7800010037001e0fe8002c
:10898c00803e20009e0f1000fcff3400f462a90012
:10899c000000eb00000f7800010037001e0fe8000c
:1089ac00803e20009e0f1000fcff3400efff3700cc
:1089bc000800fa00300798000000eb001007980040
:1089cc00e40047001000200054fa07000000e0000b
:1089dc003f003200ce409000100020006cfa0700df
:1089ec004e409000ed4f500003003a00a1c0b30080
:1089fc001000200066fa07004e409000ed4f50002a
:108a0c001a0032004e409000e84f50000d0032002a
:108a1c00818f8000f0042000808f500009003c0002
:108a2c00828f80004e4090008040780040102100e2
:108a3c0000004100014878000200e800808f8800a7
:108a4c0006003700808f80000000e0000300340037
:108a5c00808f80000000e900808f8800be009000ad
:108a6c000040eb008048780019003700100020000f
:108a7c0010079800818f80004010210080804000fa
:108a8c000040eb00804878000000eb00000f7800fd
:108a9c000a0037001e007800800078003e0090002d
:108aac00008140009e0078004010210000804000b2
:108abc0010407800004978001e0fe800808f80007d
:108acc009e0f1000f3ff34000000eb00808f880035
:108adc001e0090000080fa00000006002600fa003c
:108aec00881f78000e80e800c1022a0011000900de
:108afc00311878004002b10030c0b3006eeeb70000
:108b0c00f0e6200001052a00040009003158780025
:108b1c0020c1b30074eeb700e2e6200011c0b30030
:108b2c0050052a009dfe07006100200050052a0018
:108b3c003f01070012c0b3008000eb005f0007008c
:108b4c000000eb00000f7800200037001e007800ba
:108b5c008e80e8000000400060807800e2e6200093
:108b6c008040eb008dfe07001e0478001e0078008c
:108b7c008e80e800000040006080780073e40700fd
:108b8c00000178001e0078008e80e8000000400094
:108b9c006080780082007800250107008040780012
:108bac00401d210000004400014878009e00780020
:108bbc00401d210000804000104078000041eb0077
:108bcc009e0078003d0007001e0fe8000001200009
:108bdc009e0f1000ddff36004f0478000080fa0075
:108bec00000006000200fa00881f7800318f800018
:108bfc00408f8000008f4000408f8000308f8800b5
:108c0c001e007800408f88004100200060fd290084
:108c1c00070107000041eb009e00780027000700c9
:108c2c004000200061f5070000047800510020008e
:108c3c0030012a00fe0007000041eb00880078009c
:108c4c001e0007005000200058f5070000047800b3
:108c5c005100200090012a00f50007000041eb00b4
:108c6c008800780015000700600020004ff5070011
:108c7c000004780051002000f0012a00ec000700ed
:108c8c000041eb00880078000c0007007000200009
:108c9c0046f50700000478005100200050022a001d
:108cac00e30007000041eb00880078000300070098
:108cbc004f0478000080fa00000006000a00fa0059
:108ccc004047980031079800024f98004e409000a2
:108cdc000080fb004300de000080fb0010079800c2
:108cec004e4090008080fb001e0090004300dd0091
:108cfc0000805000670f10004e4090000080fb0079
:108d0c008000400000af200000804000be009000ba
:108d1c00010878000e4890000080fb0060004000c5
:108d2c00e10f50000f003e009e0190009e0090004d
:108d3c0000cf2000008040001040780000417800f7
:108d4c000e4890008080fb001e0078000008dd00bb
:108d5c00004069008040780000cf20000080410076
:108d6c00014878000080fa00000006000a00fa00b2
:108d7c004047980031079800420798004e409000f9
:108d8c000080fb004300de000080fb001007980011
:108d9c004e4090008080fb001e0090004300dd00e0
:108dac0000805000670f10003e0090000000e000b3
:108dbc00080032004e4090000080fb008000400014
:108dcc0000af200000804000900078003e00900032
:108ddc00010878004e0090000000e0000a0032000c
:108dec009e00900000cf20000080400010407800d2
:108dfc008080fb001e0078000088de00e1406000ef
:108e0c004e009000014878000080fa000000060037
:108e1c000000fa006382a9006362a9006342a90002
:108e2c006322a9006302a90062e2a90062c2a90040
:108e3c0062a2a800212620009140780030ceb30019
:108e4c0000c0600062e2b70062c2bf003040b300f5
:108e5c0062e2b70065e2a90065c2a90065a2a9009b
:108e6c006422a9006402a90061e2a800811f7800b5
:108e7c00821f7800831f7800217420006204200078
:108e8c0073052000824878008348780042c7a90007
:108e9c00cf0178004f017800cf007800c16a200024
:108eac009140780000ccb30000c06000d040b3000b
:108ebc00ace6b700c16d20009140780000ccb30047
:108ecc0000c060007040b300dce6b700216d2000ec
:108edc009140780000ccb30000c060000034a000ca
:108eec00d2e6b700811f7800821f7800831f7800bc
:108efc002174200062042000730520008248780051
:108f0c008348780042c7a800cf0178004f01780051
:108f1c00cf0078000080fa00000006000200fa0082
:108f2c00004f78001e80fb004013880060c2bf0019
:108f3c00614060000004e000fcff32000040eb00e8
:108f4c00004f7800401380000080fa0000000600fb
:108f5c001800fa00100f98006000b8007007980015
:108f6c00010f98000000eb00600798001e089000ad
:108f7c00e70f5000050036007e0090008e08900030
:108f8c00200f9800310f980025003700ee0090005c
:108f9c006008200000807000600798001e08900098
:108fac00c600dd006e0090000100700060079800a4
:108fbc0060c2a800000000006e009000d7ff070000
:108fcc00000000000040eb00d4ff070050079800a1
:108fdc000040eb00d1ff0700400798000040eb0079
:108fec00ceff070030079800de00900021079800a4
:108ffc002e0090004800dd0020079800ce00900065
:10900c00f00f2000808060002e00900001007000a6
:10901c00200798006000b800200f9800310f9800ce
:10902c002e089000be0890000080fa000000060098
:10903c000800fa0020079800310798000040eb0068
:10904c00204798000000eb00000f78000d0037005f
:10905c002e4090000081fb009e0078002e009000b6
:10906c0000804000104078000000fb008000690088
:10907c0060f7200000804000904078002147980065
:10908c001e0fe8003e0090009e0f1000f0ff39000c
:10909c002e4090000080fb000080fa0000000600cb
:1090ac000000fa00908f80000000e00001003a0000
:1090bc00ff3ffc00908f80000000e800908f88003c
:1090cc000080fa00000006000000fa00908f80007b
:1090dc000000e900908f8800908f80000000e00075
:1090ec0001003a000000fc000080fa0000000600bd
:00000001FF
